:040000002DEF23F0CD
:1041D50000C642899E89801200016E01C073FF12DC
:1041E5000001C088F002C089F0120072B202D0014D
:1041F5000E1200000E12000650036E010E15EC2182
:10420500F005C003F0010E15EC21F01200026E6FEF
:10421500CF01F0A49E6C9E02C06FFF6CBE1200A47D
:10422500BE1200FDD7046E04B002D08A9801D08A70
:10423500888A9A035009EC21F08A8A12000001202D
:10424500EE32F08851D9268951DA2201C0DEFF020B
:10425500C0DDFF1200000120EE30F08851D926891B
:1042650051DA2201C0DEFF02C0DDFF1200046E89B3
:104275009004501F0B200945EC21F0035045EC211B
:10428500F089801200016E000E026E01C06FFF6D95
:10429500B0A4AEFDD7A49E6FCF02F0025012000469
:1042A5006E04C007F001C006F002C005F005C001AC
:1042B500F006C002F007C003F01200C6500F0B084D
:1042C5000AD8B404D0C6500F0B0B0AD8B4C586C79C
:1042D500A0FED7C9501200036E000E026E3A0E03FF
:1042E5006005D02F0E036402D0010E026E02C001DC
:1042F500F001301200015002100310D8B406D000AE
:104305000E011A000E021A800E031A01C001F002F6
:10431500C002F003C003F012000DC001F00EC00290
:10432500F0036A8E0E046E000E056E00EC26F00199
:10433500C00DF002C00EF003C00FF0120001C0F670
:10434500FF02C0F7FFF86A000120EE21F08851D97D
:10435500268951DA220C0E0900F5CFDEFFE806FBAF
:10436500E2120001500302F3CF05F0F4CF06F0018D
:10437500500402F350062602500302F350062605A8
:10438500C001F006C002F0120007C005F008C00623
:10439500F090EC22F00009D8A409D009C005F00A74
:1043A500C006F0AEEC22F00009D8B402D0010E121E
:1043B50000000E12000150021003100410D8B408BA
:1043C500D0000E011A000E021A000E031A800E0408
:1043D5001A01C001F002C002F003C003F004C004DA
:1043E500F01200020E036E050E39EC21F0070E03E4
:1043F5006E060E39EC21F0030E036E110E39EC2119
:10440500F0000E00018C6F4B0E036E000E39EC218F
:10441500F0898E12008990610E45EC21F0096E0736
:10442500C001F008C002F007C003F008C004F003A3
:104435000E056EEBEC22F08980400E036E070E39F7
:10444500EC21F009501200000E056E000E046E00FE
:104455000E056E000E046E0AD0150E036EC60EE82C
:104465002EFED7032EFCD700D0044A052A0150049E
:104475005C02500558D8B01200EFD7000E056E004B
:104485000E046E000E056E000E046E0AD0150E03A6
:104495006EC60EE82EFED7032EFCD700D0044A05C3
:1044A5002A0150045C02500558D8B01200EFD7001D
:1044B5000E056E000E046E000E056E000E046E0AEB
:1044C500D0150E036EC60EE82EFED7032EFCD700C0
:1044D500D0044A052A0150045C02500558D8B01290
:1044E50000EFD74A6E42C013F043C014F044C01524
:1044F500F045C016F046C017F047C018F048C0197F
:10450500F049C01AF0210E000188251B6E000E89A6
:10451500211C6E4A50B9EC3FF01200400E055C01BB
:104525000E0658D8A002D0010E12002B0E036E0005
:104535000E15EC21F00650036E010E15EC21F00569
:10454500C003F0010E15EC21F02C0E036E000E15C4
:10455500EC21F0000E1200065004E1F00E055CD8C7
:10456500A002D0010E12002A0E036E000E15EC21DA
:10457500F00650036E010E15EC21F005C003F001A5
:104585000E15EC21F02C0E036E000E15EC21F0003B
:104595000E120013C00BF014C00CF015C00DF01670
:1045A500C00EF017C00FF018C010F088C0D9FF89F1
:1045B500C0DAFFDECF19F0DDCF1AF001D812000501
:1045C50000FA6E1950FD6E1A50FE6EFF6AFA50120F
:1045D50000000E066E18D00650010DF3500124D9C7
:1045E5006EF4500220DA6EDF506F6E6DB0A4AEFD32
:1045F500D70650010DF3500324D96EF4500420DA88
:104605006E6FCFDFFF062A0550065CD8B01200E3B7
:10461500D70BC011F00CC012F0111E121E114A1258
:104625002A3F0E11240B6E010E12200C6E0BC007D3
:10463500F00CC008F00DC009F00EC00AF0C7EC215F
:10464500F00009D8A412000FC005F010C006F0FE56
:10465500EC20F01200D50EF66E410EF76E000EF846
:104665006E0900F5CFEFF10900F5CFF0F10900F57E
:10467500CFF1F101EEF2F016EE40F0EE6AE550E111
:1046850050FCE1E250FAE100EE60F0730EEE6AE8EC
:1046950006FDE10001B3EF49F0000E4D1A000E4E84
:1046A5001A000E4F1A800E501A49C035F04AC0360E
:1046B500F04BC037F04CC038F04DC039F04EC03A21
:1046C500F04FC03BF050C03CF082EC38F035C049AB
:1046D500F036C04AF037C04BF038C04CF01200AE8F
:1046E500CF07F0AECF07F0AECF07F0AECF07F000A3
:1046F5000E096E000E086E12D09EA8FED708500156
:1047050024056E09500220066E05C0F6FF06C0F7A7
:10471500FFF86A0800F5CFADFF084A092A035008DB
:104725005C04500958D8B01200E7D7000E166E0089
:104735000E176E000E186E000E196E0EA008D01220
:10474500501626135017221450182215501922D826
:10475500901236133614361536D890113210320FA2
:10476500320E320E500F1010101110D8A4E6D716C5
:10477500C00EF017C00FF018C010F019C011F012DC
:1047850000000E146E000E136E000E166E000E1550
:104795006E000120EE02F08851D9268951DA22DE19
:1047A500CF25F0DDCF26F0FF0E2524176EFF0E2650
:1047B50020186E20EE04F08851D9268951DA22DEC0
:1047C500CF27F0DDCF28F0FF0E2724196EFF0E2826
:1047D500201A6E23C01BF024C01CF065EC28F012D3
:1047E50000010E106E400E0F6E000E0E6EF00E0DD7
:1047F5006E000E086E000E076E000E0A6E000E09A2
:104805006EC7EC21F00009D8A4120012D00BC00528
:10481500F00CC006F0FEEC20F00F06D8A010060F35
:1048250028F5E11028D8A4F2D7010E106E400E0F1E
:104835006E0D06D8A00E060D28EFE10E28D8B4128D
:1048450000EBD7F8EC20F00009D8A4FBD702C0F69E
:10485500FF03C0F7FF000EF86E0F0EF76403D008D4
:1048650000F55005D0F6CFE9FFF7CFEAFFEF50EF9F
:10487500EC20F00250046E0350056E024A032A0430
:10488500C0F6FF05C0F7FF000EF86E0F0EF76403C4
:10489500D00800F55005D0F6CFE9FFF7CFEAFFEFD6
:1048A500500009D8B41200CDD712501310141015AA
:1048B50010D8B424D0010E166E06D0D89012361337
:1048C5003614361536162A15AEF8D712500E5C1367
:1048D500500F581450105815501158D8A008D01220
:1048E500500E5E13500F5A1450105A1550115AD8C5
:1048F500901532143213321232162EE7D70EC00E2F
:10490500F00FC00FF010C010F011C011F01200032D
:104915006EC69EC9CF02F0C9CF02F003C0C9FFC65B
:10492500BE1200C6500F0B080AD8B40CD0C6500FE3
:104935000B0B0AD8B407D0C6889EA6FED7C7B412FB
:1049450000C7501200C6500F0B080AD8B405D0C6D0
:10495500500F0B0B0AD8A41200C7B0FED7C7A4038B
:10496500D0016A012A01D0016AC5501F0B01100050
:1049750009D8A4F4D7C5501200000E066E02AE0683
:10498500D0016C021ED8B0022A010E066E04AE04D8
:10499500D0036C041ED8B0042A03500410D8B418F0
:1049A500D0010E056E04D0D89003360436052A04CE
:1049B500AEFAD70350015C04500258D8A004D003C6
:1049C50050015E0450025AD89004320332052EF18C
:1049D500D70650D8B404D0016C021ED8B0022A0103
:1049E500C001F002C002F01200340E016EFF0E028B
:1049F5006E000E046E090E036E72EC23F0AECF1836
:104A0500F0000E1B6E080E1B6401D010D09EAAFE8E
:104A1500D7AECF18F01B50010D0E0EF324D96E0042
:104A25000EF420DA6E18C0DFFF1B2AECD7000E1A31
:104A35006E000E196E105019240C6E000E1A200D02
:104A45006E0CC00DF00C6A0CC019F00DC01AF011F7
:104A5500501924196E000E1A201A6E19C00AF01A80
:104A6500C00BF01200000E096E000E0A6E000E0B50
:104A75006E000E0C6E0550061007100810D8B42AEB
:104A8500D0010E0D6E06D0D89005360636073608CD
:104A9500360D2A08AEF8D7D89009360A360B360CEB
:104AA500360550015C06500258075003580850045B
:104AB50058D8A009D00550015E0650025A07500388
:104AC5005A0850045A0980D8900832073206320530
:104AD500320D2EE1D709C001F00AC002F00BC00368
:104AE500F00CC004F01200000E0C6E0AAE06D009E0
:104AF5006C0A1ED8B00A2A010E0C6E08AE06D00745
:104B05006C081ED8B0082A010E0C1A000E0E6E0095
:104B15000E0D6E09500A10D8B41CD0010E0B6E0490
:104B2500D0D89009360A360B2A0AAEFAD7D8900D96
:104B3500360E360950075C0A500858D8A005D0092A
:104B450050075E0A50085A0D80D8900A3209320B78
:104B55002EEDD70C50D8B404D00D6C0E1ED8B00E67
:104B65002A0DC007F00EC008F0120003AE16D001E2
:104B7500C007F002C008F003C009F0071E081E09AF
:104B85001E072A000E08220922000E0724016E00C6
:104B95000E0820026E800E0920036E06AE16D004A4
:104BA500C007F005C008F006C009F0071E081E0979
:104BB5001E072A000E08220922000E0724046E0093
:104BC5000E0820056E800E0920066E000E011A00E3
:104BD5000E021A800E031A000E041A000E051A8022
:104BE5000E061A0450015C0550025806500358D8A9
:104BF500B002D0D8901200D88012000450D8B40565
:104C0500D0015002100310D8A40CD0000E016E0084
:104C15000E026E000E036E1200042AD890033202B3
:104C2500320132000E0114066E000E0214076EFEEC
:104C35000E0314086E065007100810D8B40CD0ECFB
:104C4500D7042A010E0126000E0222000E0322D8E7
:104C550090033202320132000E0114066E000E027C
:104C650014076EFF0E0314086E065007100810D8BF
:104C7500B406D0E6D70406D89001360236033602CC
:104C8500BE03D0020E0460F6D704A0029ED890049D
:104C950032045003120550D8A4038E01C001F0025E
:104CA500C002F003C003F01200000E096E000E0AE8
:104CB5006E000E0B6E000E0C6E000E0D6E000E0ECD
:104CC5006E000E0F6E000E106E0DC011F00EC012AC
:104CD500F00FC013F010C014F005A020D00950113A
:104CE500260A5012220B5013220C50142201500D8B
:104CF5002602500E2203500F220450102201500D9F
:104D05005C02500E5803500F5804501058D8B00686
:104D1500D0010E1126000E122213221422D890095A
:104D2500360A360B360C3604BE0980D89001360299
:104D35003603360436D89008320732063205320576
:104D450050061007100810D8A4C7D720EE0DF000A4
:104D5500EE01F0070EDBCFEBFFE806FCE21200C523
:104D650080C5B0FED7C7A403D0046A042A01D004C5
:104D75006AC5501F0B04100009D8A4F4D7800E8A09
:104D8500EC24F0C7A403D0046A042A01D0046AC540
:104D9500501F0B04100009D8A4F4D7020E8AEC2486
:104DA500F0C7A403D0046A042A01D0046AC5501FC1
:104DB5000B04100009D8A4F4D7000E8AEC24F0C720
:104DC500A403D0046A042A01D0046AC5501F0B0449
:104DD500100009D8A4F4D7000E8AEC24F0C7A40368
:104DE500D0046A042A01D0046AC5501F0B041000C0
:104DF50009D8A4F4D7C584C5B4FED7C7A403D00485
:104E05006A042A01D0046AC5501F0B04100009D892
:104E1500B41200F3D7333434343A6E3A50D8A40977
:104E2500D0000E316E000E326E000E336E000E3461
:104E35006E120031C035F032C036F033C037F03471
:104E4500C038F0200E05D0D890383237323632359A
:104E550032E82EF9D73550396E338EFF0E3116FFF5
:104E65000E3216FF0E3316000E3416960E3A5E3AC3
:104E7500AE16D03A50800A970FD8B009D0000E313F
:104E85006E000E326E000E336E000E346E1200D8B8
:104E95009034323332323231323A3EF9D715D01F9F
:104EA5000E3A640FD0000E316E000E326E000E33D6
:104EB5006E000E346E1200D89031363236333634E9
:104EC500363A063A50D8A4F7D73950D8B408D03472
:104ED5001E331E321E316C000E3222332234223133
:104EE500C031F032C032F033C033F034C034F01288
:104EF500000BC00FF0106A116A0A340F3601E31077
:104F0500800F50166E1650D8A407D0000E096E00FB
:104F15000E0A6E000E0B6E12000EC00FF0106A1115
:104F25006A0D340F3601E310800F50176E1750D8F5
:104F3500A407D0000E096E000E0A6E000E0B6E124D
:104F450000000E136E000E146E000E156E175089BC
:104F55000F165E0BC017F00E50171A800E17160AA3
:104F65008EFF0E0916FF0E0A16000E0B160D8EFF8C
:104F75000E0C16FF0E0D16000E0E16180E126ED81C
:104F8500901336143615360C50095C0D500A580E20
:104F9500500B58D8A007D00C50095E0D500A5A0E78
:104FA500500B5A1380D89009360A360B36122EE765
:104FB500D713C001F014C002F015C003F016C004E9
:104FC500F017C005F000EC26F001C009F002C00A98
:104FD500F003C00BF01200000E216E1CAE09D01CB0
:104FE5001E1B1E1A1E196C000E1A221B221C2221C2
:104FF5008018AE09D0181E171E161E156C000E1649
:105005002217221822212A15C001F016C002F01716
:10501500C003F018C004F019C005F01AC006F01B53
:10502500C007F01CC008F057EC26F020EE22F00770
:105035000EEBCFDBFFE806FCE221A03AD026C01D2F
:10504500F027C01EF028C01FF029C020F01D1E1E2D
:105055001E1F1E201E1DC026F01EC027F01FC028C3
:10506500F020C029F022C01DF023C01EF024C01F6F
:10507500F025C020F01D1E1E1E1F1E201E1DC02255
:10508500F01EC023F01FC024F020C025F0010E2221
:1050950026000E2322242225222250231024102507
:1050A50010D8A406D0010E2626000E272228222974
:1050B5002220EE22F000EE15F0070EDBCFEBFFE825
:1050C50006FCE212001350175C1850800A1D6E147E
:1050D50050800A1D58D8B00CD017C021F018C02236
:1050E500F013C017F014C018F021C013F022C0143B
:1050F500F01550195C1A50800A1D6E1650800A1D55
:1051050058D8B00CD019C021F01AC022F015C0191A
:10511500F016C01AF021C015F022C016F0000120CB
:10512500EE3CF08851D9268951DA22DFB2120015FA
:10513500C01FF016C020F032D013C021F014C022D9
:10514500F021D021C00BF022C00CF01FC00DF020C3
:10515500C00EF01BC00FF01CC010F088C0D9FF892D
:10516500C0DAFFDECF1DF0DDCF1EF001D809D00576
:1051750000FA6E1D50FD6E1E50FE6EFF6AFA50124B
:1051850000214A222A2150175C1850800A1D6E22E0
:1051950050800A1D58D8B0D5D71F4A202A1F50194C
:1051A5005C1A50800A1D6E2050800A1D58D8A01226
:1051B50000C3D71AC01EF01F6A206A19341E3601B3
:1051C500E31F801E50216E2150D8A407D0000E1871
:1051D5006E000E196E000E1A6E12001DC01EF01F15
:1051E5006A206A1C341E3601E31F801E50266E2677
:1051F50050D8A407D0000E186E000E196E000E1AB6
:105205006E120026507B0F21261AC026F01D50264F
:105215001A800E2616198E1C8EFF0E1B16FF0E1CED
:1052250016000E1D16000E226E000E236E000E24B3
:105235006E070E256E18A006D01B5022261C502383
:10524500221D502422D8901A3219321832D8901BB8
:10525500361C361D36252EEED7090E256E18A006EE
:10526500D01B5022261C5023221D502422D8901AD0
:105275003219321832D890243223322232252EEEBA
:10528500D722C001F023C002F024C003F021C004DE
:10529500F026C005F000EC26F001C018F002C01998
:1052A500F003C01AF0120012C014F0156A166A1144
:1052B50034143601E3158014501E6E1E50D8A4090F
:1052C500D0000E106E000E116E000E126E000E1341
:1052D5006E1200170E146E10C015F011C016F012E4
:1052E500C017F01428186E04D0D89017321632154E
:1052F50032182EFAD71550196E118EFF0E1016FFA3
:105305000E1116000E121610501A6E11501B6E1249
:10531500501C6E1D6A8E0E1E5E1EAE16D01E50806F
:105325000A8F0FD8B009D0000E106E000E116E0056
:105335000E126E000E136E1200D8901D321C321B19
:10534500321A321E3EF9D715D0170E1E640FD00043
:105355000E106E000E116E000E126E000E136E1200
:1053650000D8901A361B361C361D361E061E50D820
:10537500A4F7D71950D8B408D01D1E1C1E1B1E1A21
:105385006C000E1B221C221D221AC010F01BC0111E
:10539500F01CC012F01DC013F01200C580C5B0FE90
:1053A500D7800E8AEC24F0000E026E050E016E5AAF
:1053B500EC22F0010E8AEC24F0000E026E050E01BF
:1053C5006E5AEC22F0C584C5B4FED7C7A403D00835
:1053D5006A082A01D0086AC5501F0B08100009D8B1
:1053E500A4F4D7000E026E140E016E5AEC22F0C51D
:1053F50080C5B0FED7810E8AEC24F0000E026E0542
:105405000E016E5AEC22F0000E0C6E000E0B6E6053
:10541500EC21F0086E08500B24096E000E0C200AD2
:105425006E09C00AF0096A09C00BF00AC00CF0C782
:10543500A403D0086A082A01D0086AC5501F0B08C2
:10544500100009D8A4F4D7C59AC588C5B8FED76099
:10545500EC21F0086E08500B240B6E000E0C200C8E
:105465006EC7A403D0086A082A01D0086AC5501F70
:105475000B08100009D8A4F4D7C58AC588C5B8FE9D
:10548500D7C584C5B4FED7C7A403D0086A082A01C6
:10549500D0086AC5501F0B08100009D8A4F4D70B13
:1054A500C006F00CC007F01200000E0114096E00D2
:1054B5000E02140A6E800E03140B6E7F0E04140C7C
:1054C5006E09500A100B100C10D8A408D0000E015C
:1054D5006E000E026E000E036E000E046E000E05C9
:1054E50014096E000E06140A6E800E07140B6E7FEB
:1054F5000E08140C6E09500A100B100C10D8A408D5
:10550500D0000E056E000E066E000E076E000E082A
:105515006E04AE1DD001C009F002C00AF003C00B35
:10552500F004C00CF0091E0A1E0B1E0C1E092A00F1
:105535000E0A220B220C22000E0924016E000E0A0F
:1055450020026E000E0B20036E800E0C20046E08E8
:10555500AE1DD005C009F006C00AF007C00BF00863
:10556500C00CF0091E0A1E0B1E0C1E092A000E0A8D
:10557500220B220C22000E0924056E000E0A2006BD
:105585006E000E0B20076E800E0C20086E000E01BB
:105595001A000E021A000E031A800E041A000E05D8
:1055A5001A000E061A000E071A800E081A05500179
:1055B5005C065002580750035808500458D8B002EA
:1055C500D0D8901200D8801200033404340E6E0E29
:1055D50050D8A409D0000E016E000E026E000E0315
:1055E5006E000E046E1200073408340D6E0D50D88F
:1055F500A409D0000E016E000E026E000E036E00AF
:105605000E046E1200038EFF0E0116FF0E0216FF2A
:105615000E0316000E0416078EFF0E0516FF0E0666
:1056250016FF0E0716000E0816000E096E000E0A6C
:105635006E000E0B6E000E0C6E7F0E0E5E0D50A0F2
:105645000F0E5E200E0D6ED89009360A360B360CFD
:10565500360550015C06500258075003580850049F
:1056650058D8A009D00550015E0650025A075003CC
:105675005A0850045A0980D8900136023603360478
:10568500360D2EE1D70EAE16D00E50800A9F0FD8DC
:10569500B009D0000E016E000E026E000E036E0002
:1056A5000E046E1200D8900C320B320A3209320EFB
:1056B5003EF9D715D01F0E0E640FD0000E016E00F7
:1056C5000E026E000E036E000E046E1200D89009D5
:1056D500360A360B360C360E060E50D8A4F7D70907
:1056E500C001F00AC002F00BC003F00CC004F012B8
:1056F50000C580C5B0FED7800E8AEC24F0000E02EE
:105705006E050E016E5AEC22F0000E8AEC24F000B4
:105715000E026E050E016E5AEC22F0C584C5B4FE6C
:10572500D7C7A403D0216A212A01D0216AC5501FF9
:105735000B21100009D8A4F4D7000E026E140E0137
:105745006E5AEC22F0C580C5B0FED7810E8AEC24D6
:10575500F0000E026E050E016E5AEC22F0000E25C9
:105765006E000E246E60EC21F0216E21502424225F
:105775006E000E2520236E22C023F0226A22C0244B
:10578500F023C025F0C7A403D0216A212A01D02126
:105795006AC5501F0B21100009D8A4F4D7C59AC5B6
:1057A50088C5B8FED760EC21F0216E215024242451
:1057B5006E000E2520256EC7A403D0216A212A017B
:1057C500D0216AC5501F0B21100009D8A4F4D7C5F4
:1057D5008AC588C5B8FED7C584C5B4FED7C7A40396
:1057E500D0216A212A01D0216AC5501F0B21100042
:1057F50009D8A4F4D724C00DF025C00EF08FEC21F4
:10580500F00DC010F00EC011F00FC012F056EC29CB
:10581500F010C01FF011C020F0120003C007F008FF
:105825006A096A0234073601E3088007500F6E0FD4
:1058350050D8A409D0000E016E000E026E000E03B2
:105845006E000E046E120006C007F0086A096A05AC
:1058550034073601E3088007500E6E0E50D8A409B0
:10586500D0000E016E000E026E000E036E000E04D7
:105875006E1200028EFF0E0116FF0E0216000E03B9
:1058850016058EFF0E0416FF0E0516000E061600F1
:105895000E0A6E000E0B6E000E0C6E000E0D6E7F66
:1058A5000E0F5E0E50980F0F5E180E0E6ED8900AF2
:1058B500360B360C360D360450015C055002580681
:1058C500500358D8A007D00450015E0550025A066F
:1058D50050035A0A80D8900136023603360E2EE65A
:1058E500D70FAE16D00F50800A970FD8B009D00049
:1058F5000E016E000E026E000E036E000E046E1297
:1059050000D8900D320C320B320A320F3EF9D71502
:10591500D0170E0F640FD0000E016E000E026E0040
:105925000E036E000E046E1200D8900A360B360C6C
:10593500360D360F060F50D8A4F7D70AC001F00B65
:10594500C002F00CC003F00DC004F01200096E098E
:1059550050D8A404AE1AD001C005F002C006F00369
:10596500C007F004C008F0051E061E071E081E0528
:105975002A000E06220722082205C00BF006C00CDD
:10598500F007C00DF008C00EF008D001C00BF00202
:10599500C00CF003C00DF004C00EF001500210035E
:1059A500100410D8A409D0000E016E000E026E007E
:1059B5000E036E000E046E1200960E0A6E06D00AD5
:1059C5002AD8900E320D320C320B32000E0B140514
:1059D5006E000E0C14066E000E0D14076EFE0E0EF4
:1059E50014086E0550061007100810D8B40DD0E73E
:1059F500D70A2A010E0B26000E0C220D220E22D8E4
:105A0500900E320D320C320B32000E0B14056E0067
:105A15000E0C14066E000E0D14076EFF0E0E140804
:105A25006E0550061007100810D8B407D0E1D70A44
:105A350006D8900B360C360D360E360DBE03D00249
:105A45000E0A60F5D70AB008D0FF0E0B16FF0E0C34
:105A5500167F0E0D16FF0E0E16D8900A320AC005D7
:105A6500F0066A076A086A05C008F0076A066A054B
:105A75006A05500B1206500C1207500D1208500EF5
:105A8500120950D8A404AE01D00E8E0BC001F00C43
:105A9500C002F00DC003F00EC004F012000DC0D915
:105AA500FF0EC0DAFFDE6ADE6ADE6ADD6ADD52DD20
:105AB50052DECF14F0DECF15F0DECF16F0DECF17B5
:105AC500F014C018F015C019F016C01AF017C01B55
:105AD500F009500A100B100C10D8A40AD020EE14AF
:105AE500F000EE01F0070EDBCFEBFFE806FCE2125B
:105AF50000210E0F6E06D0D89009360A360B360CEB
:105B0500360F2A0CAEF8D7000E106E000E116E007F
:105B15000E126E000E136ED890183619361A361BF3
:105B25003617BE1880D89014361536163617360532
:105B350050095C06500A5807500B5808500C58D8A5
:105B4500A017D00950051834E10A50061831E10BA9
:105B55005007182EE10C500818D8A42AD01050016F
:105B65005C115002581250035813500458D8A02005
:105B7500D00950055E0A50065A0B50075A0C5008BA
:105B85005A1050015C11500258125003581350041A
:105B950058D8B005D00506000E065A075A085A10FF
:105BA50050015E1150025A1250035A1350045A14F0
:105BB50080D890133212321132103209B0138ED8B8
:105BC500900C320B320A3209320F2EA5D70DC0D9EF
:105BD500FF0EC0DAFF01C0DEFF02C0DEFF03C0DE3C
:105BE500FF04C0DEFF20EE14F000EE01F0070EDB2F
:105BF500CFEBFFE806FCE21200000E2E6E27AE0981
:105C0500D0271E261E251E246C000E25222622279F
:105C1500222E8223AE3CD020C02AF021C02BF022B8
:105C2500C02CF023C02DF02A1E2B1E2C1E2D1E2A43
:105C3500C020F02BC021F02CC022F02DC023F01C79
:105C4500C02AF01DC02BF01EC02CF01FC02DF02A5D
:105C55001E2B1E2C1E2D1E2AC01CF02BC01DF02C29
:105C6500C01EF02DC01FF0010E1C26000E1D221EA9
:105C7500221F221C501D101E101F10D8A406D00173
:105C85000E2026000E212222222322030E2E26205C
:105C9500EE1CF000EE01F0070EDBCFEBFFE806FC93
:105CA500E224C009F025C00AF026C00BF027C00C7D
:105CB500F028C00DF029C00EF051EC2DF020EE2F8C
:105CC500F0070EEBCFDBFFE806FCE22EA021D02883
:105CD500C0D9FF29C0DAFFDECF2AF0DECF2BF0DEF8
:105CE500CF2CF0DECF2DF02A1E2B1E2C1E2D1E2AAA
:105CF5002A000E2B222C222D2228C0D9FF29C0DAFA
:105D0500FF2AC0DEFF2BC0DEFF2CC0DEFF2DC0DE6C
:105D1500FF2EA23AD033C02AF034C02BF035C02C68
:105D2500F036C02DF02A1E2B1E2C1E2D1E2AC03328
:105D3500F02BC034F02CC035F02DC036F02FC02A22
:105D4500F030C02BF031C02CF032C02DF02A1E2BC4
:105D55001E2C1E2D1E2AC02FF02BC030F02CC0315A
:105D6500F02DC032F0010E2F26000E3022312232E6
:105D7500222F50301031103210D8A406D0010E3326
:105D850026000E34223522362220EE2FF000EE1C9E
:105D9500F0070EDBCFEBFFE806FCE2120029C02D71
:105DA500F02E6A2F6A28342D3601E32E802D5032CD
:105DB5006E2CC02DF02E6A2F6A2B342D3601E32E62
:105DC500802D50316E3250D8B40BD03150325CD862
:105DD500B00ED03250000831242D6E180E2D6407F8
:105DE500D02AC027F02BC028F02CC029F012003192
:105DF50050D8B40BD03250315CD8B00ED0315000F1
:105E05000832242D6E180E2D6407D027C027F028E0
:105E1500C028F029C029F01200060E306E29BE30C8
:105E25008E2CBE308C288EFF0E2716FF0E281600EE
:105E35000E29162B8EFF0E2A16FF0E2B16000E2C82
:105E4500163150325CD8B01BD0D8902A362B362C60
:105E550036310632503118D8B40DD0300630C02D49
:105E6500F0070E2D16D8B406D0EFD7D890293228D2
:105E7500322732322A31503218D8B41FD0F6D732F1
:105E850050315CD8B01AD0D890273628362936320A
:105E95000632503118D8B40DD0300630C02DF00779
:105EA5000E2D16D8B406D0EFD7D8902C322B322A27
:105EB50032312A31503218D8A4F7D730AE0CD0FF82
:105EC5000E271AFF0E281AFF0E291A010E27260083
:105ED5000E2822000E292230AC0CD0FF0E2A1AFF04
:105EE5000E2B1AFF0E2C1A010E2A26000E2B22004D
:105EF5000E2C22000E306E27502A2628502B2229E0
:105F0500502C222CAE0ED0FF0E2A1AFF0E2B1AFF94
:105F15000E2C1A010E2A26000E2B22000E2C220111
:105F25000E306E2AC001F02BC002F02CC003F032F7
:105F3500C004F030C005F000EC26F001C027F002E7
:105F4500C028F003C029F012000B6EC580C5B0FE55
:105F5500D7C7A403D0086A082A01D0086AC5501F0C
:105F65000B08100009D8A4F4D7EE0E8AEC24F0C76C
:105F7500A403D0086A082A01D0086AC5501F0B0877
:105F8500100009D8A4F4D71E0E8AEC24F0C7A40388
:105F9500D0086A082A01D0086AC5501F0B081000EE
:105FA50009D8A4F4D7C584C5B4FED7C7A403D008BF
:105FB5006A082A01D0086AC5501F0B08100009D8C5
:105FC500A4F4D7000E026E140E016E26EC22F0C565
:105FD50080C5B0FED7C7A403D0086A082A01D00837
:105FE5006AC5501F0B08100009D8A4F4D7EE0E8A15
:105FF500EC24F0C7A403D0086A082A01D0086AC5B2
:10600500501F0B08100009D8A4F4D70B508AEC24B4
:10601500F0C7A403D0086A082A01D0086AC5501F32
:106025000B08100009D8A4F4D7C584C5B4FED7C79A
:10603500A403D0086A082A01D0086AC5501F0B08B6
:10604500100009D8A4F4D7000E026E140E016E26B6
:10605500EC22F0C580C5B0FED7C7A403D0086A08F6
:106065002A01D0086AC5501F0B08100009D8A4F4EE
:10607500D7EF0E8AEC24F0C7A403D0086A082A01DA
:10608500D0086AC5501F0B08100009D8A4F4D70022
:106095000E026E140E016E26EC22F0000E0D6E003F
:1060A5000E0C6E60EC21F0086E08500C24096E0091
:1060B5000E0D200A6E09C00AF0096A09C00CF00A23
:1060C500C00DF0C7A403D0086A082A01D0086AC524
:1060D500501F0B08100009D8A4F4D7C59AC588C568
:1060E500B8FED760EC21F0086E08500C240C6E0049
:1060F5000E0D200D6EC7A403D0086A082A01D0082A
:106105006AC5501F0B08100009D8A4F4D7C59AC555
:1061150088C5B8FED7C584C5B4FED7C7A403D008C3
:106125006A082A01D0086AC5501F0B08100009D853
:10613500A4F4D70CC006F00DC007F012004BC05DEB
:10614500F04CC05EF04DC058F04EC059F0FDD04F38
:10615500C0F6FF50C0F7FF000EF86E0F0EF7640390
:10616500D00800F55005D0F6CFE9FFF7CFEAFFEFED
:10617500505F6E4F4A502A000120EE28F08851D911
:10618500268951DA225F50536E546ADE50535CDE25
:10619500505458D8A0D9D020EE2AF08851D9268954
:1061A50051DA22DECF51F0DDCF52F05F50515C0065
:1061B5000E5258D8A0C9D00A0E5F18D8A40BD0200B
:1061C500EE02F08851D9268951DA22DECF5DF0DD65
:1061D500CF5EF0BAD020EE2CF08851D9268951DA5D
:1061E50022DE50DE10D8A40BD020EE24F08851D941
:1061F500268951DA22DECF5AF0DDCF5BF02AD02096
:10620500EE28F08851D9268951DA22DECF51F0DD0A
:10621500CF52F0511E521E514A522A5F50536E54AE
:106225006A515053265250542220EE2CF08851D9F1
:10623500268951DA22DECF55F0DDCF56F053505581
:1062450024D96E54505620DA6EDF50576E57505A87
:106255006E5B6A5AC05CF05C505D24516E000E5E48
:1062650020526EFF0E536EFF0E546E20EE02F08824
:1062750051D9268951DA22DECF55F0DDCF56F053BC
:10628500505526545056225150555C5650800A5749
:106295006E5250800A5758D8B021D04BC05DF04C93
:1062A500C05EF020EE26F08851D9268951DA22DE2B
:1062B500CF51F0DDCF52F020EE2FF08851D926894D
:1062C50051DA22DF50536E546A53BE54065150536F
:1062D500265250542253505826545059225DC042DC
:1062E500F05EC043F058C044F059C045F020EE3090
:1062F500F08851D9268951DA22DECF46F0DDCF4725
:10630500F020EE32F08851D9268951DA22DECF48C5
:10631500F0DDCF49F05F5074EC22F0000120EE2E45
:10632500F08851D9268951DA22DF50516E526A51CF
:10633500BE52065C50536E546A5150532652505407
:106345002253505D2654505E224FC0F6FF50C0F7D1
:10635500FF000EF86E0F0EF76403D00800F5500528
:10636500D0F6CFE9FFF7CFEAFFEF500009D8B41216
:1063750000EED6C580C5B0FED7C7A403D00A6A0A09
:106385002A01D00A6AC5501F0B0A100009D8A4F4C7
:10639500D7EE0E8AEC24F0C7A403D00A6A0A2A01B4
:1063A500D00A6AC5501F0B0A100009D8A4F4D748B3
:1063B5000E8AEC24F0C7A403D00A6A0A2A01D00A7F
:1063C5006AC5501F0B0A100009D8A4F4D7C584C5A7
:1063D500B4FED7C7A403D00A6A0A2A01D00A6AC53F
:1063E500501F0B0A100009D8A4F4D7000E026E1432
:1063F5000E016E26EC22F0C580C5B0FED7C7A403FA
:10640500D00A6A0A2A01D00A6AC5501F0B0A100071
:1064150009D8A4F4D7EE0E8AEC24F0C7A403D00A59
:106425006A0A2A01D00A6AC5501F0B0A100009D84A
:10643500A4F4D7000E8AEC24F0C7A403D00A6A0A94
:106445002A01D00A6AC5501F0B0A100009D8A4F406
:10645500D7C584C5B4FED7C7A403D00A6A0A2A01E2
:10646500D00A6AC5501F0B0A100009D8A4F4D7003A
:106475000E026E140E016E26EC22F0C580C5B0FE2C
:10648500D7C7A403D00A6A0A2A01D00A6AC5501FD1
:106495000B0A100009D8A4F4D7EF0E8AEC24F0C734
:1064A500A403D00A6A0A2A01D00A6AC5501F0B0A3A
:1064B500100009D8A4F4D7000E0E6E000E0F6E0062
:1064C5000E106E60EC21F00A6E0A500E240B6E0061
:1064D5000E0F200C6E000E10200D6E0CC00DF00B73
:1064E500C00CF00B6A0BC00EF00CC00FF00DC01005
:1064F500F0C7A403D00A6A0A2A01D00A6AC5501F48
:106505000B0A100009D8A4F4D7C59AC588C5B8FEEA
:10651500D760EC21F00A6E0A500E240B6E000E0FA8
:10652500200C6E000E10200D6E0CC00DF00BC00C73
:10653500F00B6A0BC00EF00CC00FF00DC010F0C7C9
:10654500A403D00A6A0A2A01D00A6AC5501F0B0A99
:10655500100009D8A4F4D7C59AC588C5B8FED76078
:10656500EC21F00A6E0A500E240E6E000E0F200F5D
:106575006E000E1020106EC7A403D00A6A0A2A0105
:10658500D00A6AC5501F0B0A100009D8A4F4D7C554
:106595008AC588C5B8FED7C584C5B4FED7C7A403C8
:1065A500D00A6A0A2A01D00A6AC5501F0B0A1000D0
:1065B50009D8A4F4D70E50066E0F50076E10500878
:1065C5006E096A1200346E6D0E3464B5D0000E0A81
:1065D5006E0A0E096E000E046E640E036E34C00161
:1065E500F0026ABFEC24F001C007F002C008F076A3
:1065F500EC25F0D89007360836D8900736083624AB
:106605000E0726000E0822FF0E0724F66EAD0E08B3
:1066150020F76EF86A000EF8220900F5CF13F0098D
:1066250000F5CF14F00900F5CF15F00A00F5CF16E7
:10663500F0000E0A6E640E096E34C007F0086A7623
:10664500EC25F0D89007360836D890073608364836
:106655000E0726000E0822FF0E0724F66EAD0E0863
:1066650020F76EF86A000EF8220900F5CF0FF00941
:1066750000F5CF10F00900F5CF11F00A00F5CF12A3
:10668500F020EC3AF00FC030F010C031F011C032FC
:10669500F012C033F0000E046E0A0E036E34C00112
:1066A500F0026ABFEC24F0D89001360236D890018A
:1066B500360236FF0E0124F66EAD0E0220F76EF897
:1066C5006A000EF8220900F5CF13F00900F5CF1482
:1066D500F00900F5CF15F00A00F5CF16F030C00F20
:1066E500F031C010F032C011F033C012F020EC3A96
:1066F500F00FC02CF010C02DF011C02EF012C02FDD
:10670500F02CC00FF02DC010F02EC011F02FC012CC
:10671500F0000E136E000E146E000E156E3F0E1671
:106725006E20EC3AF00FC028F010C029F011C02AF5
:10673500F012C02BF012000A0E346471D0000E0462
:106745006E0A0E036E34C001F0026ABFEC24F0D865
:106755009001360236D89001360236FF0E0124F636
:106765006EAD0E0220F76EF86A000EF8220900F5EC
:10677500CF13F00900F5CF14F00900F5CF15F00A95
:1067850000F5CF16F0000E0A6E0A0E096E34C0072A
:10679500F0086A76EC25F0D89007360836D89007C9
:1067A500360836240E0726000E0822FF0E0724F6AB
:1067B5006EAD0E0820F76EF86A000EF8220900F596
:1067C500CF0FF00900F5CF10F00900F5CF11F00A51
:1067D50000F5CF12F020EC3AF00FC030F010C031C8
:1067E500F011C032F012C033F030C00FF031C010DC
:1067F500F032C011F033C012F0000E136E000E140B
:106805006E000E156E3F0E166E20EC3AF00FC02886
:10681500F010C029F011C02AF012C02BF01200347C
:1068250050040DFF0EF324F66EAD0EF420F76EF84E
:106835006A000EF8220900F5CF0FF00900F5CF1018
:10684500F00900F5CF11F00A00F5CF12F0000E1394
:106855006E000E146E000E156E3F0E166E20EC3A8D
:10686500F00FC028F010C029F011C02AF012C02B7B
:10687500F012000450800B0D6E04500424186E03B2
:10688500BE18801850D8B40DD01828D8A408D00048
:106895000E016E000E026E000E036E000E046E03F6
:1068A5008E06D0000E016E000E026E000E036E0005
:1068B5000E046E0850800B0D1A08500824196E0737
:1068C500BE19801950D8B40DD01928D8A408D00005
:1068D5000E056E000E066E000E076E000E086E07A2
:1068E5008E06D0000E056E000E066E000E076E00B9
:1068F5000E086E0550061007100810D8A415D00014
:106905000E016E000E026E000E036E000E046E8008
:106915000E03127F0E041201C001F002C002F00343
:10692500C003F004C004F012001850D8A411D00020
:106935000E016E000E026E000E036E000E046E0157
:10694500C001F002C002F003C003F004C004F0125D
:10695500001950096E0A6A091E0A1E094A0A2A18F0
:10696500500B6E0C6A09500B260A500C227F0E0B39
:1069750024126E000E0C20136E01C00EF002C00F23
:10698500F003C010F004C011F0000E016E000E02FD
:106995006E000E036E000E046E000E146E000E15D2
:1069A5006E000E166E000E176E000E196E28D019A9
:1069B50050D8B411D0D8900E360F3610361136D8BF
:1069C50090013602360336043617BE0180D890147E
:1069D5003615361636173605500E5C06500F580715
:1069E50050105808501158D8A009D0178C05500ED2
:1069F5005E06500F5A0750105A0850115A192A1995
:106A05000E1964D5D70E500F1010101110D8B411EF
:106A1500D014800FD0D890013602360336043617CD
:106A2500BE0180D89014361536163617361206D89C
:106A3500A0130603AEEFD7000E196E17AE16D0FFE2
:106A45000E1414096EFF0E15140A6EFF0E16140BA4
:106A55006E7F0E17140C6E09500A100B100C10D80F
:106A6500A402D001A002D0010E196E1950D8B41F8E
:106A7500D0010E0126000E02220322042204A017D3
:106A8500D001C009F002C00AF003C00BF004C00C2D
:106A9500F00C340C320B320A32093209C001F00A0B
:106AA500C002F00BC003F00CC004F0124A132A1305
:106AB500BE10D0135003E11228D8A00BD0000E133E
:106AC5006E1268000E016E000E026E000E036E005F
:106AD5000E046E13BE05D0135011E11204D8B00E8A
:106AE500D0000E136E000E126E000E016E000E0227
:106AF5006E000E036E000E046E000E0D6E12C018B1
:106B0500F018A002D0038E01D0039ED8901830044F
:106B15006E0D50041201C001F002C002F003C00363
:106B2500F004C004F0120001C0D9FF02C0DAFF036F
:106B3500C0DEFF04C0DDFF20EE02F00150D92602C1
:106B450050DA2205C0DEFF06C0DDFF20EE04F001AD
:106B550050D9260250DA2207C0DEFF08C0DDFF202B
:106B6500EE15F00150D9260250DA22040EDE6E0031
:106B75000EDD6E20EE17F00150D9260250DA220400
:106B85000EDE6E000EDD6EFF0E096EFF0E0A6E2024
:106B9500EE02F00150D9260250DA22DECF0BF0DDED
:106BA500CF0CF020EE15F00150D9260250DA22DE86
:106BB500CF0DF0DDCF0EF00D1E0E1E0D4A0E2A0B69
:106BC500500D260C500E2209500D260A500E22207B
:106BD500EE19F00150D9260250DA220DC0DEFF0E63
:106BE500C0DDFFFF0E096EFF0E0A6E20EE04F001F8
:106BF50050D9260250DA22DECF0BF0DDCF0CF02083
:106C0500EE15F00150D9260250DA22DECF0DF0DD67
:106C1500CF0EF00D1E0E1E0D4A0E2A0B500D260C22
:106C2500500E2209500D260A500E2220EE1BF001AF
:106C350050D9260250DA220DC0DEFF0EC0DDFF203E
:106C4500EE19F00150D9260250DA2210EE11F001AA
:106C550050E1260250E222DECFE6FFDDCFE5FF2040
:106C6500EE1BF00150D9260250DA2210EE13F00186
:106C750050E1260250E222DECFE6FFDDCFE5FF2020
:106C8500EE2EF00150D9260250DA22010EDF6E20D9
:106C9500EE2FF00150D9260250DA22010EDF6E20C8
:106CA500EE21F00150D9260250DA22000EDE6E00E8
:106CB5000EDD6E20EE26F00150D9260250DA2200B4
:106CC5000EDE6E000EDD6E20EE24F00150D9260298
:106CD50050DA22000EDE6E000EDD6E20EE28F00189
:106CE50050D9260250DA22000EDE6E000EDD6E202F
:106CF500EE2AF00150D9260250DA22000EDE6E008F
:106D05000EDD6E20EE2CF00150D9260250DA22005D
:106D15000EDE6E000EDD6E20EE34F00150D9260237
:106D250050DA225D0EDE6E5C0EDD6E20EE30F00177
:106D350050D9260250DA22FF0EDE6EFF0EDD6E20E0
:106D4500EE32F00150D9260250DA22000EDE6E0036
:106D55000EDD6E20EE0BF00150D9260250DA22002E
:106D65000EDE6E000EDD6E20EE0DF00150D926020E
:106D750050DA22000EDE6E000EDD6E20EE0FF00101
:106D850050D9260250DA22000EDE6E000EDD6E00AE
:106D95000E0F6E020E0F6401D028D00F50030D3771
:106DA5000EF326000EF422F3500124D96EF450029E
:106DB50020DA6E000EDE6E000EDD6E0F50030D370D
:106DC5000EF326000EF42201C009F002C00AF0F30A
:106DD500500926F4500A22020E0924D96E000E0A23
:106DE50020DA6E000EDF6E0F2AD4D701C088F002BC
:106DF500C089F01200C580C5B0FED7C7A403D00A6C
:106E05006A0A2A01D00A6AC5501F0B0A100009D860
:106E1500A4F4D7EE0E8AEC24F0C7A403D00A6A0ABC
:106E25002A01D00A6AC5501F0B0A100009D8A4F41C
:106E3500D71E0E8AEC24F0C7A403D00A6A0A2A01D9
:106E4500D00A6AC5501F0B0A100009D8A4F4D7C58B
:106E550084C5B4FED7C7A403D00A6A0A2A01D00A9A
:106E65006AC5501F0B0A100009D8A4F4D7000E02FA
:106E75006E140E016E26EC22F0C580C5B0FED7C794
:106E8500A403D00A6A0A2A01D00A6AC5501F0B0A50
:106E9500100009D8A4F4D7EE0E8AEC24F0C7A40399
:106EA500D00A6A0A2A01D00A6AC5501F0B0A1000C7
:106EB50009D8A4F4D7580E8AEC24F0C7A403D00A45
:106EC5006A0A2A01D00A6AC5501F0B0A100009D8A0
:106ED500A4F4D7C584C5B4FED7C7A403D00A6A0AEB
:106EE5002A01D00A6AC5501F0B0A100009D8A4F45C
:106EF500D7000E026E140E016E26EC22F0C580C579
:106F0500B0FED7C7A403D00A6A0A2A01D00A6AC507
:106F1500501F0B0A100009D8A4F4D7EE0E8AEC24F2
:106F2500F0C7A403D00A6A0A2A01D00A6AC5501F0D
:106F35000B0A100009D8A4F4D7000E8AEC24F0C778
:106F4500A403D00A6A0A2A01D00A6AC5501F0B0A8F
:106F5500100009D8A4F4D7C584C5B4FED7C7A403C7
:106F6500D00A6A0A2A01D00A6AC5501F0B0A100006
:106F750009D8A4F4D7000E026E140E016E26EC2279
:106F8500F0C580C5B0FED7C7A403D00A6A0A2A0196
:106F9500D00A6AC5501F0B0A100009D8A4F4D7EF10
:106FA5000E8AEC24F0C7A403D00A6A0A2A01D00A83
:106FB5006AC5501F0B0A100009D8A4F4D7000E02A9
:106FC5006E140E016E26EC22F0000E0F6E000E10F0
:106FD5006E000E116E000E126E60EC21F00A6E0A44
:106FE500500F240B6E000E10200C6E000E11200D9C
:106FF5006E000E12200E6E0DC00EF00CC00DF00BC3
:10700500C00CF00B6A0BC00FF00CC010F00DC011D6
:10701500F00EC012F0C7A403D00A6A0A2A01D00AEA
:107025006AC5501F0B0A100009D8A4F4D7C59AC524
:1070350088C5B8FED760EC21F00A6E0A500F240B04
:107045006E000E10200C6E000E11200D6E000E123B
:10705500200E6E0DC00EF00CC00DF00BC00CF00B29
:107065006A0BC00FF00CC010F00DC011F00EC0126D
:10707500F0C7A403D00A6A0A2A01D00A6AC5501FBC
:107085000B0A100009D8A4F4D7C59AC588C5B8FE5F
:10709500D760EC21F00A6E0A500F240F6E000E1017
:1070A50020106E000E1120116E000E1220126EC7F8
:1070B500A403D00A6A0A2A01D00A6AC5501F0B0A1E
:1070C500100009D8A4F4D7C58AC588C5B8FED7C5A8
:1070D50084C5B4FED7C7A403D00A6A0A2A01D00A18
:1070E5006AC5501F0B0A100009D8A4F4D70FC006B3
:1070F500F010C007F011C008F012C009F0120038F6
:1071050050800B456E38503824476E37BE47804750
:1071150050D8B40DD04728D8A408D0000E356E003D
:107125000E366E000E376E000E386E378E06D000A6
:107135000E356E000E366E000E376E000E386E3C44
:1071450050800B466E45504618D8A4458C3C503CA3
:1071550024466E3BBE46804650D8B40DD04628D84E
:10716500A408D0000E396E000E3A6E000E3B6E007C
:107175000E3C6E3B8E06D0000E396E000E3A6E0048
:107185000E3B6E000E3C6E4750465CD8B022D04593
:10719500AC02D0800E451A47C048F046C047F048BB
:1071A500C046F035C048F039C035F048C039F03632
:1071B500C048F03AC036F048C03AF037C048F03B16
:1071C500C037F048C03BF038C048F03CC038F04804
:1071D500C03CF0000E486E47503D6E3E6A3D1E3E77
:1071E5001E3D4A3E2A46503F6E406A3D503F263E70
:1071F50050402240BE2CD0405004E11A0E3F5CD8CE
:10720500A026D03550361037103810D8B402D0012A
:107215000E01D0000E486E000E356E000E366E0063
:107225000E376E000E386E46C047F015D048A005E3
:10723500D0D89048300109486E02D0D890483235F0
:10724500B0488E38343832373236323532472A46EE
:1072550050475CD8A0EBD745BC29D04750D8A409E6
:10726500D0000E356E000E366E000E376E000E38ED
:107275006E1200395035263A5036223B5037223CA3
:1072850050382238A083D048A006D0D8904832483C
:10729500500109486E02D0D890483235B0488E3832
:1072A500343832373236323532472A70D039503594
:1072B5005C3A5036583B5037583850800A3D6E3C42
:1072C50050800A3D58D8B036D035C03DF036C03E66
:1072D500F037C03FF038C040F03D1E3E1E3F1E4017
:1072E5001E3D2A000E3E223F22402239503D2441B8
:1072F5006E3A503E20426E3B503F20436E3C50401C
:1073050020446EFF0E4124356EFF0E4220366EFF7F
:107315000E4320376EFF0E4420386E800E451A4806
:107325006C4850D8A40FD0010E3526000E362237F2
:1073350022382208D03950355E3A50365A3B5037FC
:107345005A3C50385A3550361037103810D8A41CCE
:10735500D04850D8A419D0000E356E000E366E00F8
:107365000E376E000E386E1200D890353636363729
:1073750036383648BE358048A002D0D88001D0D8EE
:107385009048364750D8A4470637AEEED7000E468C
:107395006E48AE0AD048C03DF07F0E3D16D8A40217
:1073A500D035A002D0010E466E4650D8B420D0018B
:1073B5000E3526000E36223722382238A018D03551
:1073C500C03DF036C03EF037C03FF038C040F04019
:1073D5003440323F323E323D323DC035F03EC0365C
:1073E500F03FC037F040C038F04728D8A4472A47B7
:1073F50028D8B403D04750D8A40DD0000E356E0060
:107405000E366E000E376E000E386E4750D8A40249
:10741500D0000E456E47A002D0378E01D0379ED8DA
:10742500904730386E45BE388E35C035F036C0369B
:10743500F037C037F038C038F012001250800B1BFF
:107445006E12501224216E11BE21802150D8B40D28
:10745500D02128D8A408D0000E0F6E000E106E00A3
:107465000E116E000E126E118E08D0000E0F6E00FA
:107475000E106E000E116E000E126E1650800B1B54
:107485001A16501624206E15BE20802050D8B40D33
:10749500D02028D8A408D0000E136E000E146E005C
:1074A5000E156E000E166E158E08D0000E136E00AA
:1074B5000E146E000E156E000E166E2050D8B40315
:1074C500D02150D8A409D0000E0F6E000E106E000A
:1074D5000E116E000E126E120015500F02F3CF261C
:1074E500F0F4CF27F026501C6E1D6A1E6A1F6A270E
:1074F50050226E236A246A256A14501002F3CF269F
:10750500F0F4CF27F026501C26000E1D221E221F48
:107515002227502226000E23222422252213501131
:1075250002F3CF26F0F4CF27F026501C26000E1DBF
:10753500221E221F2227502226000E232224222526
:10754500221EC01FF01DC01EF01CC01DF01C6A13BA
:10755500501002F3CF26F0F4CF27F026501C262733
:10756500501D22000E1E22000E1F2214500F02F382
:10757500CF26F0F4CF27F026501C2627501D2200D9
:107585000E1E22000E1F221EC01FF01DC01EF01C65
:10759500C01DF01C6A13500F02F3CF26F0F4CF275D
:1075A500F026501C2627501D22000E1E22000E1FFD
:1075B5002215501002F3CF26F0F4CF27F0265022E3
:1075C5002627502322000E2422000E2522145011B6
:1075D50002F3CF26F0F4CF27F0265022262750239A
:1075E50022000E2422000E252215501102F3CF266B
:1075F500F0F4CF27F02650176E2750186E196A1A27
:107605006A19C01AF018C019F017C018F0176A17D0
:1076150050222618502322195024221A5025221CA4
:10762500C017F01DC018F01EC019F01FC01AF019C0
:107635000E05D0D8901A32193218321732E82EF9C1
:10764500D71750222618502322195024221A5025C4
:10765500221EC01FF01DC01EF01CC01DF01C6A209C
:107665005021C017F0186A1726000E1822820E172F
:1076750024266EFF0E1820276E0FD0D890223623B1
:1076850036243625361FBE2280D8901C361D361E60
:10769500361F362606D8A0270624AEEFD7000E20C3
:1076A5006E1FAE16D0FF0E1C14176EFF0E1D14189C
:1076B5006EFF0E1E14196E7F0E1F141A6E175018CA
:1076C5001019101A10D8A402D022A002D0010E2041
:1076D5006E2050D8B41FD0010E2226000E2322247E
:1076E50022252225A017D022C017F023C018F02488
:1076F500C019F025C01AF01A341A32193218321787
:107705003217C022F018C023F019C024F01AC02582
:10771500F0264A272A27BE0DD0275003E12628D870
:10772500A008D0000E226E000E236E800E246E7F00
:107735000E20D027BE05D027500EE12604D8B00B69
:10774500D0000E226E000E236E000E246E000E2554
:107755006E000E1B6E0FD026C021F0FF0E2216FF05
:107765000E23167F0E2416000E251621B0248ED862
:10777500902130256E1B50251222C00FF023C0101A
:10778500F024C011F025C012F01200CB0E036E00DC
:107795000E15EC21F0390E036E010E15EC21F02CBF
:1077A5000E036E010E15EC21F0000E036E010E1591
:1077B500EC21F0340E036E010E15EC21F0020E03E0
:1077C5006E010E15EC21F0CF0E036E000E15EC21A7
:1077D500F0000E036E010E15EC21F0C10E036E01D3
:1077E5000E15EC21F0300E036E010E15EC21F0E8BC
:1077F5000E036E000E15EC21F0850E036E010E15BD
:10780500EC21F0000E036E010E15EC21F0780E034D
:107815006E010E15EC21F0EA0E036E000E15EC213B
:10782500F0000E036E010E15EC21F0000E036E0143
:107835000E15EC21F0ED0E036E000E15EC21F06433
:107845000E036E010E15EC21F0030E036E010E15ED
:10785500EC21F0120E036E010E15EC21F0810E03E2
:107865006E010E15EC21F0F70E036E000E15EC21DE
:10787500F0200E036E010E15EC21F0C00E036E0014
:107885000E15EC21F0230E036E010E15EC21F0C14F
:107895000E036E000E15EC21F0100E036E010E1591
:1078A500EC21F0C50E036E000E15EC21F03E0E0323
:1078B5006E010E15EC21F0280E036E010E15EC215C
:1078C500F0C70E036E000E15EC21F0860E036E0157
:1078D5000E15EC21F0360E036E000E15EC21F08826
:1078E5000E036E010E15EC21F03A0E036E000E1517
:1078F500EC21F0550E036E010E15EC21F0B10E03CF
:107905006E000E15EC21F0000E036E010E15EC2134
:10791500F0180E036E010E15EC21F0B60E036E0085
:107925000E15EC21F0080E036E010E15EC21F08208
:107935000E036E010E15EC21F0270E036E010E15D8
:10794500EC21F0F20E036E000E15EC21F0000E0393
:107955006E010E15EC21F0260E036E000E15EC21BE
:10796500F0010E036E010E15EC21F0E00E036E0022
:107975000E15EC21F00F0E036E010E15EC21F03102
:107985000E036E010E15EC21F02B0E036E010E1584
:10799500EC21F00C0E036E010E15EC21F00E0E031A
:1079A5006E010E15EC21F0080E036E010E15EC218B
:1079B500F04E0E036E010E15EC21F0F10E036E0173
:1079C5000E15EC21F0370E036E010E15EC21F007B4
:1079D5000E036E010E15EC21F0100E036E010E154F
:1079E500EC21F0030E036E010E15EC21F00E0E03D3
:1079F5006E010E15EC21F0090E036E010E15EC213A
:107A0500F0000E036E010E15EC21F0E10E036E0081
:107A15000E15EC21F0000E036E010E15EC21F00E93
:107A25000E036E010E15EC21F0140E036E010E15FA
:107A3500EC21F0030E036E010E15EC21F0110E037F
:107A45006E010E15EC21F0070E036E010E15EC21EB
:107A5500F0310E036E010E15EC21F0C10E036E011F
:107A65000E15EC21F0480E036E010E15EC21F00801
:107A75000E036E010E15EC21F00F0E036E010E15AF
:107A8500EC21F00C0E036E010E15EC21F0310E0306
:107A95006E010E15EC21F0360E036E010E15EC216C
:107AA500F00F0E036E010E15EC21F0110E036E00A2
:107AB5000E15EC21F0000E026E780E016E40EC22E0
:107AC500F02C0E036E000E15EC21F08AC00BF08B26
:107AD500C00CF0F3EC23F0290E036E000E15EC211B
:107AE500F02C0E036E000E15EC21F01200306E30F6
:107AF500AE1FD1306C3050800A120FD8A0A1D00033
:107B05000E0A6E0A0E096E000E046E640E036E30C8
:107B150050016E026A01BE0206BFEC24F001C007E7
:107B2500F002C008F076EC25F0D89007360836D874
:107B35009007360836240E0726000E0822FF0E078A
:107B450024F66EAD0E0820F76EF86A000EF82209CD
:107B550000F5CF13F00900F5CF14F00900F5CF15A6
:107B6500F00A00F5CF16F0000E0A6E640E096E30AD
:107B750050076E086A07BE080676EC25F0D8900710
:107B8500360836D89007360836480E0726000E0800
:107B950022FF0E0724F66EAD0E0820F76EF86A0078
:107BA5000EF8220900F5CF0FF00900F5CF10F00906
:107BB50000F5CF11F00A00F5CF12F020EC3AF00FE6
:107BC500C02CF010C02DF011C02EF012C02FF02CDB
:107BD500C00FF02DC010F02EC011F02FC012F00014
:107BE5000E046E0A0E036E3050016E026A01BE026B
:107BF50006BFEC24F0D89001360236D89001360243
:107C050036FF0E0124F66EAD0E0220F76EF86A00FF
:107C15000EF8220900F5CF13F00900F5CF14F0098D
:107C250000F5CF15F00A00F5CF16F020EC3AF00F6D
:107C3500C028F010C029F011C02AF012C02BF01294
:107C4500003050800A750FD8A05BD0000E0A6E0A6E
:107C55000E096E3050076E086A07BE080676EC25D9
:107C6500F0D89007360836D89007360836240E0720
:107C750026000E0822FF0E0724F66EAD0E0820F72B
:107C85006EF86A000EF8220900F5CF0FF00900F52D
:107C9500CF10F00900F5CF11F00A00F5CF12F00072
:107CA5000E046E0A0E036E3050016E026A01BE02AA
:107CB50006BFEC24F0D89001360236D89001360282
:107CC50036FF0E0124F66EAD0E0220F76EF86A003F
:107CD5000EF8220900F5CF13F00900F5CF14F009CD
:107CE50000F5CF15F00A00F5CF16F020EC3AF00FAD
:107CF500C028F010C029F011C02AF012C02BF012D4
:107D0500003050040DFF0EF324F66EAD0EF420F78F
:107D15006EF86A000EF8220900F5CF28F00900F583
:107D2500CF29F00900F5CF2AF00A00F5CF2BF01284
:107D3500003050800A120FD8A0A1D0000E0A6E0A9A
:107D45000E096E000E046E640E036E3050016E0255
:107D55006A01BE0206BFEC24F001C007F002C008AC
:107D6500F076EC25F0D89007360836D89007360817
:107D750036240E0726000E0822CB0E0724F66EAD1C
:107D85000E0820F76EF86A000EF8220900F5CF13E9
:107D9500F00900F5CF14F00900F5CF15F00A00F54C
:107DA500CF16F0000E0A6E640E096E3050076E088D
:107DB5006A07BE080676EC25F0D89007360836D84F
:107DC5009007360836480E0726000E0822CB0E0708
:107DD50024F66EAD0E0820F76EF86A000EF822093B
:107DE50000F5CF0FF00900F5CF10F00900F5CF1120
:107DF500F00A00F5CF12F020EC3AF00FC02CF0108D
:107E0500C02DF011C02EF012C02FF02CC00FF02D98
:107E1500C010F02EC011F02FC012F0000E046E0A33
:107E25000E036E3050016E026A01BE0206BFEC24DD
:107E3500F0D89001360236D89001360236CB0E01C5
:107E450024F66EAD0E0220F76EF86A000EF82209D0
:107E550000F5CF13F00900F5CF14F00900F5CF15A3
:107E6500F00A00F5CF16F020EC3AF00FC028F0101C
:107E7500C029F011C02AF012C02BF012003050803A
:107E85000A750FD8A05BD0000E0A6E0A0E096E3077
:107E950050076E086A07BE080676EC25F0D89007ED
:107EA500360836D89007360836240E0726000E0801
:107EB50022CB0E0724F66EAD0E0820F76EF86A0089
:107EC5000EF8220900F5CF0FF00900F5CF10F009E3
:107ED50000F5CF11F00A00F5CF12F0000E046E0A7E
:107EE5000E036E3050016E026A01BE0206BFEC241D
:107EF500F0D89001360236D89001360236CB0E0105
:107F050024F66EAD0E0220F76EF86A000EF822090F
:107F150000F5CF13F00900F5CF14F00900F5CF15E2
:107F2500F00A00F5CF16F020EC3AF00FC028F0105B
:107F3500C029F011C02AF012C02BF01200305004F5
:107F45000DCB0EF324F66EAD0EF420F76EF86A0035
:107F55000EF8220900F5CF28F00900F5CF29F00920
:107F650000F5CF2AF00A00F5CF2BF01200276E2777
:107F7500C040F011D0940E0DD0990E0BD0810E0992
:107F8500D09A0E07D0840E05D08E0E03D0E60E01D2
:107F9500D0F80E406E19D04050B00AD8B4F9D705C4
:107FA5000AD8B4F4D7710AD8B4EFD7120AD8B4E412
:107FB500D70A0AD8B4E5D7380AD8B4E4D7120AD80C
:107FC500B4D9D70A0AD8B4DAD720EE07F01B50D9AE
:107FD500261C50DA2240501F6E206ADE501F5CDEE0
:107FE500502058D8A0120020EE09F01B50D9261CAD
:107FF50050DA22DECF1DF0DDCF1EF040501D5C00B3
:108005000E1E58D8A0120015C02EF016C02FF02055
:10801500EE03F01B50D9261C50DA22DECF34F0DDFA
:10802500CF35F034503510D8B41200D890353234ED
:1080350032D89035323432D8903532343220EE038E
:10804500F01B50D9261C50DA22DECF1DF0DDCF1EE5
:10805500F0070E1D16000E1E161D501E10D8B40278
:10806500D0344A352A20EE0BF01B50D9261C50DAA5
:1080750022DE50DE10D8A40BD020EE03F01B50D921
:10808500261C50DA22DECF3EF0DDCF3FF02AD0208D
:10809500EE07F01B50D9261C50DA22DECF1DF0DD8D
:1080A500CF1EF01D1E1E1E1D4A1E2A40501F6E208B
:1080B5006A1D501F261E50202220EE0BF01B50D9A2
:1080C500261C50DA22DECF21F0DDCF22F01F502111
:1080D50024D96E20502220DA6EDF50236E23503EC5
:1080E5006E3F6A000120EE3FF08851D9268951DAAA
:1080F50022DFA28AD1000E256E000E266E20EE022A
:10810500F01B50D9261C50DA22DF50D8A489D02084
:10811500EE07F01B50D9261C50DA22DECF1DF0DD0C
:10812500CF1EF01D1E1E1E1D4A1E2A40501D240175
:108135006E000E1E20026E20EE05F01B50D9261C87
:1081450050DA22DECF03F0DDCF04F0B4EC21F001EC
:10815500C032F002C033F032C001F033C002F03457
:10816500C003F035C004F0B4EC21F001C03AF002D0
:10817500C03BF03C6A3D6A000E396E000E386E4316
:10818500D03EC02CF03FC02DF0000E376E000E36ED
:108195006E32D01BC0D9FF1CC0DAFFDECF1DF0DD6B
:1081A500CF1EF03A501D263B501E221DC0F6FF1E65
:1081B500C0F7FFF86A0800F5CF41F0010E3A260036
:1081C5000E3B223C223D22000E2B6E000E2A6E072E
:1081D500D0D89041322C06D8A02D062A4A2B2A2B1E
:1081E5005008E1080E2A5CD8B004D02C502D10D8C8
:1081F500A4EFD7364A372A3450365C35503758D82D
:10820500A0C8D7384A392A20EE05F01B50D9261CBC
:1082150050DA22DE50385CDE503958D8B01200B042
:10822500D720EE02F01B50D9261C50DA22DE04D8E6
:10823500A4120020EE07F01B50D9261C50DA22DECE
:10824500CF1DF0DDCF1EF01D1E1E1E1D4A1E2A402D
:10825500501D24016E000E1E20026E20EE05F01B3F
:1082650050D9261C50DA22DECF03F0DDCF04F0B45E
:10827500EC21F001C032F002C033F032C001F0331E
:10828500C002F020EE03F01B50D9261C50DA22DE86
:10829500CF03F0DDCF04F0B4EC21F001C03AF002D9
:1082A500C03BF03C6A3D6A000E396E000E386E9F89
:1082B500D0000E376E000E366E74D01BC0D9FF1C71
:1082C500C0DAFFDECF1DF0DDCF1EF03A501D263B94
:1082D500501E221DC0F6FF1EC0F7FFF86A0800F504
:1082E500CF41F0010E3A26000E3B223C223D2200F2
:1082F5000E1D6EFF0E1E6E000E1714016EFF0E187A
:1083050014026E41C003F0046AB4EC21F001C01FF1
:10831500F002C020F04150216E226A211E221E214A
:108325004A222A000E2124016E010E2220026E002F
:108335000E1914036EFF0E1A14046EB4EC21F0012D
:10834500501F260250202220C01FF0206A1D501FFA
:10835500161E5020164150236E246A231E241E2308
:108365004A242A000E2324016E010E2420026E19D0
:1083750050036E046AB4EC21F0175041020150F32A
:10838500260250F422F4CFF3FFF46AFF0EF3160031
:108395000EF4161F50F310286E2050F410296E3677
:1083A5004A372A3E50365C3F503758D8A086D720EA
:1083B500EE03F01B50D9261C50DA22DECF1DF0DD6E
:1083C500CF1EF03EC01FF03FC020F01F1E201E1F15
:1083D5004A202A1D501F261E5020221F503A2620B3
:1083E500503B22000E3C22000E3D22384A392A20FD
:1083F500EE05F01B50D9261C50DA22DE50385CDE23
:10840500503958D8B0120054D720EE02F01B50D97D
:10841500261C50DA22DF50D8A4CBD020EE07F01B63
:1084250050D9261C50DA22DECF1DF0DDCF1EF01DFF
:108435001E1E1E1D4A1E2A40501D24016E000E1EC2
:1084450020026E20EE05F01B50D9261C50DA22DEE4
:10845500CF03F0DDCF04F0B4EC21F001C032F0021F
:10846500C033F032C001F033C002F034C003F03540
:10847500C004F0B4EC21F001C03AF002C03BF03C7E
:108485006A3D6A000E396E000E386E85D013C03015
:10849500F014C031F03EC02CF03FC02DF0000E3777
:1084A5006E000E366E6ED01BC0D9FF1CC0DAFFDE23
:1084B500CF1DF0DDCF1EF03A501D263B501E221D6C
:1084C500C0F6FF1EC0F7FFF86A0800F5CF41F001BE
:1084D5000E3A26000E3B223C223D22000E2B6E005A
:1084E5000E2A6E43D041A019D030C00BF031C00C1C
:1084F500F02EC00DF02FC00EF017C00FF018C010F1
:10850500F088C0D9FF89C0DAFFDECF1DF0DDCF1EB0
:10851500F001D822D00500FA6E18D030C00BF0312A
:10852500C00CF02EC00DF02FC00EF019C00FF01AC0
:10853500C010F088C0D9FF89C0DAFFDECF1DF0DD9D
:10854500CF1EF001D809D00500FA6E1D50FD6E1E34
:1085550050FE6EFF6AFA501200D8904132304A310F
:108565002A2C06D8A02D062A4A2B2A2B5008E108CA
:108575000E2A5CD8B004D02C502D10D8A4B3D73611
:108585004A372A3450365C35503758D8A08CD72E08
:108595004A2F2A384A392A20EE05F01B50D9261CC5
:1085A50050DA22DE50385CDE503958D8B012006EF1
:1085B500D720EE02F01B50D9261C50DA22DE04D853
:1085C500A4120020EE07F01B50D9261C50DA22DE3B
:1085D500CF1DF0DDCF1EF01D1E1E1E1D4A1E2A409A
:1085E500501D24016E000E1E20026E20EE05F01BAC
:1085F50050D9261C50DA22DECF03F0DDCF04F0B4CB
:10860500EC21F001C032F002C033F032C001F0338A
:10861500C002F020EE03F01B50D9261C50DA22DEF2
:10862500CF03F0DDCF04F0B4EC21F001C03AF00245
:10863500C03BF03C6A3D6A000E396E000E386EC6CE
:10864500D013C030F014C031F0000E376E000E3676
:108655006E95D01BC0D9FF1CC0DAFFDECF1DF0DD43
:10866500CF1EF03A501D263B501E221DC0F6FF1EA0
:10867500C0F7FFF86A0800F5CF41F0010E3A260071
:108685000E3B223C223D22000E1D6EFF0E1E6E008B
:108695000E1714016EFF0E1814026E41C003F0048C
:1086A5006AB4EC21F001C01FF002C020F041502156
:1086B5006E226A211E221E214A222A000E21240131
:1086C5006E010E2220026E000E1914036EFF0E1AA3
:1086D50014046EB4EC21F001501F26025020222014
:1086E500C01FF0206A1D501F161E50201641502332
:1086F5006E246A231E241E234A242A000E232401E5
:108705006E010E2420026E1950036E046AB4EC212A
:10871500F0175041020150F3260250F422F4CFF332
:10872500FFF46AFF0EF316000EF4161F50F310281F
:108735006E2050F410296E30C00BF031C00CF02EB5
:10874500C00DF02FC00EF028C00FF029C010F08822
:10875500C0D9FF89C0DAFFDECF1DF0DDCF1EF001E5
:10876500D809D00500FA6E1D50FD6E1E50FE6EFF35
:108775006AFA501200304A312A364A372A3E5036B4
:108785005C3F503758D8A065D720EE03F01B50D971
:10879500261C50DA22DECF1DF0DDCF1EF03EC01FB5
:1087A500F03FC020F01F1E201E1F4A202A1D501F0B
:1087B500261E5020221F503A2620503B22000E3CF8
:1087C50022000E3D222E4A2F2A384A392A20EE054C
:1087D500F01B50D9261C50DA22DE50385CDE5039A9
:1087E50058D8B012002DD7550E0001DD6F000EDEF2
:1087F5006F9EEF49F0250EF319D8B40AD051C0D9B0
:10880500FF52C0DAFFF3C0DFFF514A522A9EEF49FB
:10881500F0000EEA6F000EE96F000EF06F000EEF2C
:108825006F04D00001EF85534A542A53C0F6FF5414
:10883500C0F7FFF86A0800F550300AD8B4F2D753EC
:10884500C0F6FF54C0F7FFF86A0800F5506EEC213A
:10885500F0D8A036D0000E0001EA6F000EE96FE9EE
:10886500C001F0EAC002F0000E046E0A0E036EB4F9
:10887500EC21F001C0E9F002C0EAF0D00E0001D30E
:108885006FFF0ED46F53C0F6FF54C0F7FFF86A08A8
:1088950000F550D56FD66BD351D527D451D623D5F6
:1088A50051E927D651EA23534A542A53C0F6FF54B7
:1088B500C0F7FFF86A0800F5506EEC21F0D8B0CF8C
:1088C500D753C0F6FF54C0F7FFF86A0800F5502EDD
:1088D5000AD8A432D00001F08D534A542A000EF272
:1088E5006F000EF16F1DD0F1C001F0F2C002F00073
:1088F5000E046E0A0E036EB4EC21F053C0F6FF545D
:10890500C0F7FFF86A0800F5500126000E0222D0D4
:108915000E01240001F16FFF0E0220F26F534A543D
:108925002A53C0F6FF54C0F7FFF86A0800F5506EE9
:10893500EC21F0D8A00ED0D7D7000E0001F26F00C1
:108945000EF16FF08906D0EF8904D0F08523D0EFC2
:108955008D21D053C0F6FF54C0F7FF534A542AF86F
:108965006A0800F5CFF3F00001F351000AD8B4AC62
:10897500EF49F0640AD8B40ED0020AD8B4E6D70F8E
:108985000AD8B408D0050AD8B4DED7190AD8B4DF96
:10899500D79EEF49F0070EF015D8B45DD3F0A904C2
:1089A500D0000EF26F060EF16FDDC0D9FFDEC0DA22
:1089B500FFDECFEBF0DECFECF0DECFEDF0DECFEE7D
:1089C500F0040EDD27000EDE23EEAF15D0EBC0015F
:1089D500F0ECC002F0EDC003F0EEC004F0DDEC21D8
:1089E500F001C0EBF002C0ECF003C0EDF004C0EE06
:1089F500F0030E0001EF13000EE46F000EE36FEBC2
:108A050051EC11ED11EE11D8B482D0ED35EE358271
:108A15000FE36FE46BFF0EE423E307D8A0E407E35D
:108A2500C001F0E4C002F0000E046E030E036EB444
:108A3500EC21F001C0E3F002C0E4F0E3C007F0E48C
:108A4500C008F0000E0A6E0A0E096E76EC25F007D6
:108A5500C0E3F008C0E4F00001E4AF03D0E307D8B9
:108A6500A0E407E351000879EC3DF028C0DFF029C8
:108A7500C0E0F02AC0E1F02BC0E2F0DFC00FF0E06B
:108A8500C010F0E1C011F0E2C012F0EBC013F0EC41
:108A9500C014F0EDC015F0EEC016F020EC3AF00F62
:108AA500C0DFF010C0E0F011C0E1F012C0E2F0DF6D
:108AB500C001F0E0C002F0E1C003F0E2C004F00044
:108AC5000E056E000E066E800E076E3F0E086E5781
:108AD500EC2AF0D8B005D00001E307D8A0E40717C9
:108AE500D0DFC001F0E0C002F0E1C003F0E2C00455
:108AF500F0000E056E000E066E200E076E410E0884
:108B05006E57EC2AF0D8A003D00001E34BE42B000C
:108B150001F2BF06D0F25121E10D0EF15DD8B01D75
:108B2500D0EBC035F0ECC036F0EDC037F0EEC03814
:108B3500F0F151E5EC32F028C039F029C03AF02ABD
:108B4500C03BF02BC03CF082EC38F035C0EBF03682
:108B5500C0ECF037C0EDF038C0EEF00001E4BF0620
:108B6500D0E45123E10A0EE35DD8B01FD0EB51EC00
:108B750011ED11EE11D8B464D0EBC031F0ECC03278
:108B8500F0EDC033F0EEC034F00DEC27F03150328B
:108B95001033103410D8A454D00001E4BF51D0E4F0
:108BA5005104E1020EE35DD8A04BD0DFC001F0E037
:108BB500C002F0E1C003F0E2C004F05F0E056E7084
:108BC5000E066E890E076E400E086E57EC2AF0D819
:108BD500B003D00001F70E02D00001F80EE327FF25
:108BE5000EE423E35179EC3DF028C0DFF029C0E025
:108BF500F02AC0E1F02BC0E2F0EBC001F0ECC002BE
:108C0500F0EDC003F0EEC004F0DFC005F0E0C006F3
:108C1500F0E1C007F0E2C008F0E7EC2AF001C0E59A
:108C2500F002C0E6F003C0E7F004C0E8F0000E0073
:108C350001EB6F000EEC6F000EED6F000EEE6F3C5A
:108C4500D0EBC031F0ECC032F0EDC033F0EEC03403
:108C5500F00DEC27F031C0E5F032C0E6F033C0E7A7
:108C6500F034C0E8F0EBC049F0ECC04AF0EDC04B81
:108C7500F0EEC04CF0E5C001F0E6C002F0E7C0033D
:108C8500F0E8C004F0000EA9EC2CF001C04DF00294
:108C9500C04EF003C04FF004C050F04FEC23F04934
:108CA500C0EBF04AC0ECF04BC0EDF04CC0EEF0006C
:108CB5000E0001E46F000EE36F010EF36F0A0EF371
:108CC50019D8B41BD0F351040D330EF324F66EAE50
:108CD5000EF420F76EF86A000EF8220900F550E54B
:108CE5005D0900F550E6590900F550E7590900F509
:108CF50050E859D8A002D0F32BE1D7F3C0D3F0D474
:108D05006BD3BFD407F151D327F251D423E351D309
:108D150027E451D423D351E95FD451EA5BF151F2F1
:108D250011D8B403D0E907D8A0EA07030EEF15D38D
:108D35006F000EF015D46FD351D411D8B403D0E918
:108D450007D8A0EA07EFA531D0030EEF15D36F00C2
:108D55000EF015D46FD351D411D8B414D051C0D955
:108D6500FF52C0DAFF2D0EDF6E514A522A0BD05149
:108D7500C0D9FF52C0DAFF300EDF6E514A522AE9E0
:108D850007D8A0EA07EABF75D0EA51F1E1E905D8AD
:108D9500A070D0EDD751C0D9FF52C0DAFF200EDF49
:108DA5006E514A522AE907D8A0EA07EABF05D0EA78
:108DB50051F1E1E905D8B0EED7030EEF15D36F00F9
:108DC5000EF015D46FD351D411D8B453D051C0D9A6
:108DD500FF52C0DAFF2D0E4AD0E5C001F0E6C00211
:108DE500F0E7C003F0E8C004F0F351040D330EF3CF
:108DF50024F66EAE0EF420F76EF86A000EF822091E
:108E050000F5CF05F00900F5CF06F00900F5CF070D
:108E1500F00A00F5CF08F035EC25F001C0DFF002CF
:108E2500C0E0F003C0E1F004C0E2F0DFC00EF0E006
:108E3500C00FF0E1C010F0E2C011F00A0E126E0092
:108E45000E136E000E146E000E156E57EC24F00E08
:108E5500C0DFF00FC0E0F010C0E1F011C0E2F0009B
:108E650001DF51300F51C0D9FF52C0DAFFDF6E511B
:108E75004A522AF307F329D8B40CD0AED751C0D93A
:108E8500FF52C0DAFF300EDF6E514A522AE307D88F
:108E9500A0E407E4BF05D0E451F1E1E305D8B0EE65
:108EA500D7F2BF09D0F25104E1090EF15DD8A00354
:108EB500D0080EF36F02D0F1C0F3F0F351F15F006B
:108EC5000EF3BFFF0EF25BF351D8B408D051C0D9F1
:108ED500FF52C0DAFF2E0EDF6E514A522AF3517946
:108EE500EC3DF028C0D9F029C0DAF02AC0DBF02B20
:108EF500C0DCF0EBC013F0ECC014F0EDC015F0EEE3
:108F0500C016F0D9C00FF0DAC010F0DBC011F0DCEC
:108F1500C012F020EC3AF00FC031F010C032F01161
:108F2500C033F012C034F00DEC27F031C0E5F0325B
:108F3500C0E6F033C0E7F034C0E8F077D0E5C00113
:108F4500F0E6C002F0E7C003F0E8C004F00001F36A
:108F550051040D330EF324F66EAE0EF420F76EF8C1
:108F65006A000EF8220900F5CF05F00900F5CF06D5
:108F7500F00900F5CF07F00A00F5CF08F035EC252C
:108F8500F001C0DFF002C0E0F003C0E1F004C0E290
:108F9500F0DFC00EF0E0C00FF0E1C010F0E2C0114C
:108FA500F00A0E126E000E136E000E146E000E15F2
:108FB5006E57EC24F00EC0DFF00FC0E0F010C0E1FA
:108FC500F011C0E2F00001DF51300F51C0D9FF525E
:108FD500C0DAFFDF6E514A522AE5C00EF0E6C00F37
:108FE500F0E7C010F0E8C011F0F351040D330EF3B3
:108FF50024F66EAE0EF420F76EF86A000EF822091C
:1090050000F5CF12F00900F5CF13F00900F5CF14E4
:10901500F00A00F5CF15F057EC24F00EC0E5F00F7F
:10902500C0E6F010C0E7F011C0E8F00001F307F367
:1090350029D8B40CD083D751C0D9FF52C0DAFF303C
:109045000EDF6E514A522AF107D8A0F207F151F20C
:1090550011D8B471D1F0D7EFBD2ED0EFA90ED0DD68
:10906500C0D9FFDEC0DAFFDECFE5F0DECFE6F0DE09
:10907500CFE7F0DECFE8F0040E0ED0DDC0D9FFDE7D
:10908500C0DAFFDECFE5F0DDCFE6F0000EE6BFFF8C
:109095000EE76FE86F020EDD27000EDE23E8AF2D29
:1090A500D0030EEF13E81FE71FE61FE56D000EE680
:1090B50023E723E82322D0EFA90ED0DDC0D9FFDEB8
:1090C500C0DAFFDECFE5F0DECFE6F0DECFE7F0DE9B
:1090D500CFE8F0040E0FD0DDC0D9FFDEC0DAFFDE29
:1090E500CFD3F0DDCFD4F0D3C0E5F0D4C0E6F0E7C0
:1090F5006BE86B020EDD27000EDE23F151F211D86D
:10910500A408D0E551E611E711E811D8A402D0F181
:109115004BF22B010EF36F0A0EF319D8B41BD0F3E3
:1091250051040D330EF324F66EAE0EF420F76EF8EF
:109135006A000EF8220900F550E55D0900F550E6D4
:10914500590900F550E7590900F550E859D8A0022A
:10915500D0F32BE1D7800EF3BF7F0ED36FF151F320
:109165005DF251800AD359D8B003D0F1C0F3F010A5
:10917500D0F251800AD36FF351F15D800EF3BF7FBA
:109185000ED359D8B005D0F351F16FF26BF1BFF2A0
:1091950007E951EA11D8B40DD0030EEF15D36F00CE
:1091A5000EF015D46FD351D411D8B403D0E907D834
:1091B500A0EA07F0AD13D0E951F15DF251800AD371
:1091C5006FEA51800AD359D8B005D0F151E95FF261
:1091D50051EA5B04D0000EEA6F000EE96F800EF3D2
:1091E500BF7F0ED36FE951F35DEA51800AD359D899
:1091F500B007D0F351E95F000EF3BFFF0EEA5B0441
:10920500D0000EEA6F000EE96FEFA522D0030EEF36
:1092150015D36F000EF015D46FD351D411D8B408FF
:10922500D051C0D9FF52C0DAFF2D0EDF6E514A5220
:109235002AE951EA11D8B477D051C0D9FF52C0DA22
:10924500FF300EDF6E514A522AE907D8A0EA07F02F
:10925500D7E951EA11D8B40FD051C0D9FF52C0DABD
:10926500FF200EDF6E514A522AE907D8A0EA07E926
:1092750051EA11D8A4F1D7030EEF15D36F000EF004
:1092850015D46FD351D411D8B44ED051C0D9FF5293
:10929500C0DAFF2D0EDF6E45D0F1C0D3F0F2C0D499
:1092A500F0D890D337D437D890D337D437330ED3BB
:1092B50025F66EAE0ED421F76EF86A000EF8220977
:1092C50000F5CF05F00900F5CF06F00900F5CF0749
:1092D500F00A00F5CF08F0E5C001F0E6C002F0E7BE
:1092E500C003F0E8C004F035EC25F001C00EF00233
:1092F500C00FF003C010F004C011F00A0E126E008A
:109305000E136E000E146E000E156E57EC24F00E43
:1093150050300F0001F36F51C0D9FF52C0DAFFF38F
:10932500C0DFFF514A522AF107D8A0F207F129B44C
:10933500E1F229D8A4B1D753C0F6FF54C0F7FF53C3
:109345004A542AF86A0800F5CFF3F0F351D8A4FD82
:10935500EF43F051C0D9FF52C0DAFF000EDF6E12A5
:10936500009B8CD298D388D38AD38C000E0F0138FA
:109375006F000E396F000E3A6F8A80000E926E04F0
:109385000E936E180E946EF19E938C400E616EC610
:1093950086C694C692C690C68A9F0EC86EC59A9414
:1093A5008EAC98AC94B896670EAF6EAC8AAB8EABAC
:1093B50098AECF01F1AECF01F1AB88010E6E6E0A0A
:1093C5000E6C6E6D8C6C8A900E716E7096670E7554
:1093D5006E729872947096200E726E010E026EF483
:1093E5000E016E40EC22F0C8EC3BF08D0E016E00D4
:1093F5000E026E160E036E460E046E010E066E40CC
:109405000E056E000E086EF00E076E96EC35F00137
:109415000E026EF40E016E40EC22F08D0E016E0010
:109425000E026EF3EC20F01E0E016EFF0E026EA111
:10943500EC21F0000E026E000E016E21EC21F00011
:109445000E026E1F0E016E2DEC21F0000E4C6E1EED
:109455000E4B6E000E4E6E640E4D6E9A0E4F6EFFE5
:109465000E506EA1EC30F03A0E026E980E016E4071
:10947500EC22F0000E246E000E236EC3EC23F0A246
:109485000EA7EC2FF006C06AF107C06BF1090E00BC
:1094950001F56F1E0EF46FE40EE82EFED7F42FFCD7
:1094A500D7F52FFAD700F0A40EA7EC2FF006C06C65
:1094B500F107C06DF1090E0001F56F1E0EF46FE4A2
:1094C5000EE82EFED7F42FFCD7F52FFAD700F0A61D
:1094D5000EA7EC2FF006C06EF107C06FF1090E0064
:1094E50001F56F1E0EF46FE40EE82EFED7F42FFC87
:1094F500D7F52FFAD700F0A80EA7EC2FF006C0700D
:10950500F107C071F1090E0001F56F1E0EF46FE44D
:109515000EE82EFED7F42FFCD7F52FFAD700F0AAC8
:109525000EA7EC2FF006C072F107C073F1090E000B
:1095350001F56F1E0EF46FE40EE82EFED7F42FFC36
:10954500D7F52FFAD700F0AC0EA7EC2FF006C074B4
:10955500F107C075F12B0E016EFF0E026E000E04B1
:109565006E090E036E72EC23F0ECEC20F0000E0297
:109575006E320E016E40EC22F0F4EC21F0750E0215
:109585006EFF0E036E24EC24F0000E0101DD6F3D2D
:109595000E026EFF0E036E24EC24F0110E016EFF19
:1095A5000E026EA1EC21F0070E026EE00E016E2D8B
:1095B500EC21F03B0E0101DD6502D0000EDD6FB23E
:1095C500EC26F07BEC2BF01FC076F120C077F1760E
:1095D500C10DF077C10EF08FEC21F00DC05EF10EDC
:1095E500C05FF10FC060F1000E1B6E250E1C6E43AF
:1095F5000E1D6E000E0C6E800E0D6E470E0E6E5E0D
:10960500C109F05FC10AF060C10BF07BEC27F009DE
:10961500C018F00AC019F00BC01AF0DCEC28F018DD
:10962500C027F019C028F01AC029F0000E2A6E20B4
:109635000E2B6EC20E2C6ED1EC2EF027C0ECF1284D
:10964500C0EDF129C0EEF1D0EC29F006C00DF00710
:10965500C00EF08FEC21F00DC061F10EC062F10F6C
:10966500C063F1000E0C6E800E0D6E470E0E6E611E
:10967500C109F062C10AF063C10BF07BEC27F00968
:10968500C018F00AC019F00BC01AF0000E1B6EC806
:109695000E1C6E420E1D6EDCEC28F018C0E6F119AA
:1096A500C0E7F11AC0E8F181AC5DD0000E516E0142
:1096B5000E526EE30E536EFF0E546EEEC1F7F0EDD3
:1096C500C1F6F0ECC1F5F00001F46BF4C055F0F50E
:1096D500C056F0F6C057F0F7C058F0F6EC43F0115D
:1096E5000E016EFF0E026EA1EC21F0F80E026E0067
:1096F5000E016E2DEC21F0000E4C6E140E4B6E001B
:109705000E4E6E0A0E4D6E000E4F6E010E506EA17E
:10971500EC30F0040E016EFF0E026EA1EC21F0009C
:109725000E4C6E440E4B6E000E4E6E0D0E4D6EF5CC
:109735000E4F6EFF0E506EA1EC30F0F70E016EFE6F
:109745000E026EA1EC21F0000E4C6E480E4B6E0021
:109755000E4E6E0F0E4D6EFB0E4F6EFF0E506EA130
:10976500EC30F080D0660E136E660E146EE60E15A4
:109775006E3F0E166EEEC1F7F0EDC1F6F0ECC1F5D9
:10978500F00001F46BF4C00FF0F5C010F0F6C01155
:10979500F0F7C012F020EC3AF00FC035F010C036EB
:1097A500F011C037F012C038F0000E396E000E3AD5
:1097B5006E000E3B6E420E3C6E82EC38F036C0F801
:1097C500F037C0F9F038C0FAF0F8C064F1F9C065B7
:1097D500F1FAC066F1000E516E010E526EE30E53A2
:1097E5006EFF0E546E66C1F7F065C1F6F064C1F503
:1097F500F00001F46BF4C055F0F5C056F0F6C05713
:10980500F0F7C058F0F6EC43F0110E016EFF0E02B2
:109815006EA1EC21F0F80E026E000E016E2DEC210A
:10982500F0000E4C6E140E4B6E000E4E6E0A0E4D71
:109835006E000E4F6E010E506EA1EC30F0F70E016A
:109845006EFE0E026EA1EC21F0000E4C6E480E4B22
:109855006E000E4E6E0F0E4D6EFD0E4F6EFF0E50CE
:109865006EA1EC30F0AA0E026EFF0E036E24EC24FE
:10987500F0000E026E010E036E24EC24F05B0E0266
:109885006EFF0E036E24EC24F0000E516E010E5295
:109895006EDE0E536EFF0E546EE8C1F7F0E7C1F6AB
:1098A500F0E6C1F5F00001F46BF4C055F0F5C056D3
:1098B500F0F6C057F0F7C058F0F6EC43F0110E0182
:1098C5006EFF0E026EA1EC21F0000E026E1F0E015E
:1098D5006E2DEC21F0000E4C6E5F0E4B6E000E4EA1
:1098E5006E0A0E4D6E000E4F6E010E506EA1EC30DD
:1098F500F0F70E016EFE0E026EA1EC21F0000E4C8B
:109905006E740E4B6E000E4E6E0F0E4D6EF10E4FB9
:109915006EFF0E506EA1EC30F0B90E026EFF0E0315
:109925006E24EC24F0000E026E010E036E24EC246E
:10993500F05B0E026EFF0E036E24EC24F01E0E018A
:1099450001DD19D8A440D2000EB66F000EB56F41E7
:109955000EB55D010EB659D8B01AD0B5C113F0B623
:10996500C114F0B20EB525D96E050EB621DA6EDF3B
:10997500500001F46FF451156E166A000E186E0052
:109985000E176ECCEC22F00101B54BB62BE0D700DB
:109995000EB86F000EB76F400EB75D010EB859D8FF
:1099A500B01BD0010EB7250001F46F000E0101B800
:1099B500210001F56FB20EF425D96E050EF521DAF9
:1099C5006EB20E0101B725E16E050EB821E26EDF1C
:1099D500CFE7FFB74BB82BDFD7ECC118F0EDC119B6
:1099E500F0EEC11AF0000E1B6EC80E1C6E420E1D65
:1099F5006EDCEC28F018C0ECF119C0EDF11AC0EEE0
:109A0500F1ECC101F0EDC102F0EEC103F0E00E048E
:109A15006EDA0E056E440E066EB8EC25F0D8B0076A
:109A2500D0E00E0101EC6FDA0EED6F440EEE6FC063
:109A35000E2A6EDA0E2B6EC40E2C6EECC127F0EDDD
:109A4500C128F0EEC129F0D1EC2EF027C009F0288D
:109A5500C00AF029C00BF0000E0C6E000E0D6E4012
:109A65000E0E6E7BEC27F009C0ECF10AC0EDF10B90
:109A7500C0EEF1000E016E340E026E440E036EEC64
:109A8500C104F0EDC105F0EEC106F0B8EC25F0D843
:109A9500B014D0ECC127F0EDC128F0EEC129F000DB
:109AA5000E2A6E340E2B6EC40E2C6ED1EC2EF027C2
:109AB500C0ECF128C0EDF129C0EEF1000E016EF009
:109AC5000E026E430E036EECC104F0EDC105F0EE1F
:109AD500C106F0B8EC25F0D8B014D0ECC127F0EDF4
:109AE500C128F0EEC129F0000E2A6EF00E2B6EC3D0
:109AF5000E2C6ED1EC2EF027C0ECF128C0EDF1292B
:109B0500C0EEF1000E016E700E026E430E036EEC98
:109B1500C104F0EDC105F0EEC106F0B8EC25F0D8B2
:109B2500B014D0ECC127F0EDC128F0EEC129F0004A
:109B35000E2A6E700E2B6EC30E2C6ED1EC2EF027F6
:109B4500C0ECF128C0EDF129C0EEF1ECC101F0ED5A
:109B5500C102F0EEC103F07DEC21F001C027F00257
:109B6500C028F003C029F0000E2A6E6F0E2B6E433D
:109B75000E2C6ED1EC2EF027C0ECF128C0EDF129AA
:109B8500C0EEF1ECC110F0EDC111F0EEC112F056CE
:109B9500EC29F010C0F1F6000E0101D26F000ED1D4
:109BA5006F400ED15D010ED259D8B023D0B20ED17F
:109BB50025D96E050ED221DA6EDF50D8B416D0D174
:109BC500C113F0D2C114F0B20ED125D96E050ED253
:109BD50021DA6EDF500001F46FF451156E166AF844
:109BE5000E186E000E176ECCEC22F00101D14BD28F
:109BF5002BD7D7000EBA6F000EB96F410EB95D01B4
:109C05000EBA59D8B01AD0B9C113F0BAC114F0724E
:109C15000EB925D96E040EBA21DA6EDF500001F4B3
:109C25006FF451156E166A000E186E000E176ECC85
:109C3500EC22F00101B94BBA2BE0D7000EBC6F0046
:109C45000EBB6F400EBB5D010EBC59D8B01BD001D9
:109C55000EBB250001F46F000E0101BC210001F5CA
:109C65006F720EF425D96E040EF521DA6E720E01AF
:109C750001BB25E16E040EBC21E26EDFCFE7FFBB21
:109C85004BBC2BDFD7E6C118F0E7C119F0E8C11AC4
:109C9500F0000E1B6EC80E1C6E420E1D6EDCEC280D
:109CA500F018C0E6F119C0E7F11AC0E8F1E6C10104
:109CB500F0E7C102F0E8C103F0480E046E9C0E0502
:109CC5006E450E066EB8EC25F0D8B007D0480E01EB
:109CD50001E66F9C0EE76F450EE86F400E2A6E9CFD
:109CE5000E2B6EC50E2C6EE6C127F0E7C128F0E8F5
:109CF500C129F0D1EC2EF027C009F028C00AF029BF
:109D0500C00BF0000E0C6E700E0D6E410E0E6E7BCC
:109D1500EC27F009C0E6F10AC0E7F10BC0E8F1E66F
:109D2500C101F0E7C102F0E8C103F07DEC21F001CB
:109D3500C027F002C028F003C029F0000E2A6E6F7C
:109D45000E2B6E430E2C6ED1EC2EF027C0E6F128BB
:109D5500C0E7F129C0E8F1E6C110F0E7C111F0E86C
:109D6500C112F056EC29F010C0B1F5000E0101D476
:109D75006F000ED36F400ED35D010ED459D8B023BA
:109D8500D0720ED325D96E040ED421DA6EDF50D8E9
:109D9500B416D0D3C113F0D4C114F0720ED325D9A3
:109DA5006E040ED421DA6EDF500001F46FF4511504
:109DB5006E166A000E186E1F0E176ECCEC22F0019F
:109DC50001D34BD42BD7D7AB8EAB98AECF78F1AEB2
:109DD500CF78F1AECF78F1AECF78F1AB88F7EC2440
:109DE500F00AC0DBF10BC0DCF1000E516E010E5222
:109DF5006EED0E536EFF0E546EDBC155F0DCC15691
:109E0500F0F6EC43F0110E016EFF0E026EA1EC218F
:109E1500F0FF0E026EE00E016E2DEC21F0000E4CEF
:109E25006EFC0E4B6E000E4E6E0A0E4D6E000E4F02
:109E35006E010E506EA1EC30F0F70E016EFE0E02B3
:109E45006EA1EC21F0010E4C6E240E4B6E000E4EF1
:109E55006E0F0E4D6EF40E4F6EFF0E506EA1EC3070
:109E6500F0010E4C6E2F0E4B6E000E4E6E130E4D06
:109E75006EF90E4F6EFF0E506EA1EC30F0D00E0253
:109E85006EFF0E036E24EC24F0000E026E010E032D
:109E95006E24EC24F05B0E026EFF0E036E24EC24A0
:109EA500F01E0E0101DD19D8A4AFD0000EBE6F0063
:109EB5000EBD6F410EBD5D010EBE59D8B01AD0BDA5
:109EC500C113F0BEC114F0F20EBD25D96E060EBE4B
:109ED50021DA6EDF500001F46FF451156E166A0039
:109EE5000E186E000E176ECCEC22F00101BD4BBEB4
:109EF5002BE0D7000EC06F000EBF6F400EBF5D0197
:109F05000EC059D8B01BD0010EBF250001F46F005B
:109F15000E0101C0210001F56FF20EF425D96E0680
:109F25000EF521DA6EF20E0101BF25E16E060EC0B7
:109F350021E26EDFCFE7FFBF4BC02BDFD7910EDBF2
:109F45005D010EDC59D8B004D0010EDC6F910EDB3B
:109F55006F700E0001F46FFE0EF56FDBC1F6F0DCDD
:109F6500C1F7F0F451F627F551F723D890F733F6FA
:109F750033D890F733F633D890F733F633F6C0DBA2
:109F8500F1F7C0DCF1DBC1F4F0DCC1F5F0F41FF54D
:109F95001FF44BF52BEF0EF4250101DB6F000E00CE
:109FA50001F5210101DC6F28EE31F0DBC1DFFF0097
:109FB5000ED66F000ED56F400ED55D010ED659D861
:109FC500B023D0F20ED525D96E060ED621DA6EDF76
:109FD50050D8B416D0D5C113F0D6C114F0F20ED5B1
:109FE50025D96E060ED621DA6EDF500001F46FF426
:109FF50051156E166AFF0E186EE00E176ECCEC2228
:10A00500F00101D54BD62BD7D7FDEC36F006C08F26
:10A01500F107C090F108C091F109C092F101018FDB
:10A0250051901191119211D8B4F7D39205D8B0F48B
:10A03500D372510001F46F010173510001F56FF600
:10A045006BF76BF6C0F7F0F5C0F6F0F4C0F5F0F479
:10A055006BF41FF51FF61FF71FF42B000EF523F603
:10A0650023F72301018F510001F4250101CD6F90E4
:10A07500510001F5210101CE6F91510001F6210139
:10A0850001CF6F92510001F7210101D06F000E42FF
:10A095006F000E436F000E446F000E456FCDC11566
:10A0A500F0CEC116F0CFC117F0D0C118F074C119A8
:10A0B500F075C11AF01B6A1C6AEEEC27F021EE025E
:10A0C500F0070EEBCFDBFFE806FCE221EE02F00025
:10A0D500EE1CF0070EDBCFEBFFE806FCE2000E24DA
:10A0E5006E000E256E800E266E000E276E42C1286C
:10A0F500F043C129F0FFEC2DF021EE0AF0070EEB3D
:10A10500CFDBFFE806FCE2000E01017E6F000E7F4B
:10A115006F000E806F000E816FD00E0A257E6F07CF
:10A125000E0B217F6F000E0C21806F000E0D21811B
:10A135006F000E796F000E7A6F000E7B6F000E7C3C
:10A145006F81BF09D08151801167E1D00E7E5D0717
:10A155000E7F59D8B061D0CDC10EF0CEC10FF0CF72
:10A16500C110F0D0C111F0CDC112F0CEC113F0CFA6
:10A17500C114F0D0C115F098EC23F00EC046F10FD4
:10A18500C047F110C048F111C049F148C14AF14931
:10A19500C14BF101014C6B4D6B4AC1F4F04BC1F55C
:10A1A500F04CC1F6F04DC1F7F0100E06D00001D805
:10A1B50090F733F633F533F433E82EF8D7F4C07956
:10A1C500F1F5C07AF1F6C07BF1F7C07CF179C1F405
:10A1D500F07AC1F5F07BC1F6F07CC1F7F0F41FF51C
:10A1E5001FF61FF71FF42B000EF523F623F72301A7
:10A1F500017E510001F42501017E6F7F510001F5BB
:10A205002101017F6F80510001F6210101806F81DD
:10A21500510001F7210101816FBCEC31F006C093BB
:10A22500F107C094F108C095F109C096F1010193B9
:10A2350051941195119611D8B4EFD29605D8B0EC7A
:10A24500D2000E9E6F000E9F6F000EA06F000EA134
:10A255006F70C115F071C116F0176A186ACDC11972
:10A26500F0CEC11AF0CFC11BF0D0C11CF0EEEC2727
:10A27500F021EE12F0070EEBCFDBFFE806FCE22142
:10A28500EE12F000EE1CF0070EDBCFEBFFE806FC4C
:10A29500E2800E246E000E256E000E266E000E273F
:10A2A5006E9E0E286E010E296EFFEC2DF021EE1A22
:10A2B500F0070EEBCFDBFFE806FCE26CC115F06D95
:10A2C500C116F0176A186A000E196E000E1A6E0193
:10A2D5000E1B6E000E1C6EEEEC27F021EE22F00731
:10A2E5000EEBCFDBFFE806FCE201011A51222597B0
:10A2F5006F1B512321986F1C512421996F1D5125E6
:10A30500219A6F000E876F000E886F000E896F000F
:10A315000E8A6F6EC115F06FC116F0176A186ACDF7
:10A32500C119F0CEC11AF0CFC11BF0D0C11CF0EE9F
:10A33500EC27F021EE2AF0070EEBCFDBFFE806FC59
:10A34500E221EE2AF000EE1CF0070EDBCFEBFFE872
:10A3550006FCE2000E246E010E256E000E266E0030
:10A365000E276E870E286E010E296EFFEC2DF0214B
:10A37500EE32F0070EEBCFDBFFE806FCE201016AE7
:10A38500510001F46F01016B510001F56FF66BF798
:10A395006B0F0ED890F437F537F637F737E82EF907
:10A3A500D7F4C04EF1F5C04FF1F6C050F1F7C051EA
:10A3B500F101014E513225526F4F513321536F50E8
:10A3C500513421546F51513521556F93C101F0948A
:10A3D500C102F095C103F096C104F052C105F053D6
:10A3E500C106F054C107F055C108F057EC26F0211D
:10A3F500EE3AF0070EEBCFDBFFE806FCE2000E01BC
:10A40500018B6F000E8C6F000E8D6F000E8E6F210D
:10A41500EE3AF000EE1CF0070EDBCFEBFFE806FC92
:10A42500E2000E246E000E256E200E266E000E270D
:10A435006E8B0E286E010E296EFFEC2DF021EEDEDF
:10A44500F0070EEBCFDBFFE806FCE201019751DEDA
:10A455005D9851DF599951E0599A51E159D8B005A4
:10A46500D0E207000EE35BE45BE55B97C1F4F0988F
:10A47500C1F5F099C1F6F09AC1F7F00001F41FF5A6
:10A485001FF61FF71FF42B000EF523F623F7230104
:10A4950001DE510001F4250101AA6FDF510001F52C
:10A4A500210101AB6FE0510001F6210101AC6FE123
:10A4B500510001F7210101AD6FE2C1AEF1E3C1AF7A
:10A4C500F1E4C1B0F1E5C1B1F121EEAAF000EE1C55
:10A4D500F0070EDBCFEBFFE806FCE2000E246E80F2
:10A4E5000E256E000E266E000E276E9E0E286E013E
:10A4F5000E296EFFEC2DF021EEA2F0070EEBCFDB5F
:10A50500FFE806FCE2A2C101F0A3C102F0A4C10369
:10A51500F0A5C104F0640E056E000E066E000E0770
:10A525006E000E086E35EC25F001C056F102C057DD
:10A53500F103C058F104C059F1640E056E000E0612
:10A545006E000E076E000E086EA2C101F0A3C102D7
:10A55500F0A4C103F0A5C104F035EC25F001C00E4F
:10A56500F002C00FF003C010F004C011F0640E1229
:10A575006E000E136E000E146E000E156E98EC2311
:10A58500F00E1E0F1E101E111E0E2A000E0F221099
:10A595002211220101A2510E245A6FA3510F205BF3
:10A5A5006FA45110205C6FA55111205D6F000E51F5
:10A5B5006E010E526EC50E536EFF0E546E56C1558A
:10A5C500F057C156F058C157F059C158F05AC15902
:10A5D500F05BC15AF05CC15BF05DC15CF0F6EC4329
:10A5E500F0110E016EFF0E026EA1EC21F0070E02B6
:10A5F5006EE00E016E2DEC21F0000E4C6E910E4BAF
:10A605006E000E4E6E0A0E4D6E000E4F6E010E5010
:10A615006EA1EC30F0F70E016EFE0E026EA1EC217C
:10A62500F0000E4C6ED30E4B6E000E4E6E0F0E4D9F
:10A635006EE80E4F6EFF0E506EA1EC30F08A0E02E2
:10A645006EFF0E036E24EC24F0000E026E010E0365
:10A655006E24EC24F05B0E026EFF0E036E24EC24D8
:10A66500F01E0E0101DD19D8A4D7D0000EC26F006F
:10A675000EC16F410EC15D010EC259D8B01AD0C1CD
:10A68500C113F0C2C114F0320EC125D96E030EC23A
:10A6950021DA6EDF500001F46FF451156E166A0071
:10A6A5000E186E000E176ECCEC22F00101C14BC2E4
:10A6B5002BE0D7000EC46F000EC36F1AD0010EC376
:10A6C500250001F46F000E0101C4210001F56F3270
:10A6D5000EF425D96E030EF521DA6E320E0101C393
:10A6E50025E16E030EC421E26EDFCFE7FFC34BC445
:10A6F5002B400EC35D010EC459D8A0E0D7A2C1C935
:10A70500F1A3C1CAF1A4C1CBF1A5C1CCF1CC5110C3
:10A71500E1DC0EC95D7C0ECA59010ECB59D8B008D3
:10A72500D0DC0EC96F7C0ECA6F010ECB6F000ECC4C
:10A735006F240EC925016E830ECA21026EFE0ECB53
:10A7450021036EFF0ECC21046E190E056E000E0658
:10A755006E000E076E000E086E35EC25F001C0C9BF
:10A76500F102C0CAF103C0CBF104C0CCF1C9C1F4F8
:10A77500F0CAC1F5F0CBC1F6F0CCC1F7F00001F499
:10A785001FF51FF61FF71FF42B000EF523F623F711
:10A7950023EF0EF4250101C96F000E0001F521011B
:10A7A50001CA6F000E0001F6210101CB6F000E00FA
:10A7B50001F7210101CC6F24EE71F0C9C1DFFF0063
:10A7C5000ED86F000ED76F400ED75D010ED859D841
:10A7D500B023D0320ED725D96E030ED821DA6EDF1D
:10A7E50050D8B416D0D7C113F0D8C114F0320ED753
:10A7F50025D96E030ED821DA6EDF500001F46FF40F
:10A8050051156E166A070E186EE00E176ECCEC2207
:10A81500F00101D74BD82BD7D7FF0E45EC21F0011E
:10A82500017D6F00F001017DAD24D09B0E076E0107
:10A835000E086E0DEC22F00101006F800E9B19D8F9
:10A84500B418D0800E9C19D8B414D09B51D8B4112B
:10A85500D09C51D8B40ED09CC101F09DC102F09B93
:10A865005152EC21F001C0EFF102C0F0F103C0F14B
:10A87500F100F0EFC101F0F0C102F0F1C103F00009
:10A885000E046EB40E056E420E066EB8EC25F0D8B9
:10A89500B089D281AC5DD0820E516E010E526ED759
:10A8A5000E536EFF0E546EF1C1F7F0F0C1F6F0EFE6
:10A8B500C1F5F00001F46BF4C055F0F5C056F0F6A3
:10A8C500C057F0F7C058F0F6EC43F0110E016EFFDB
:10A8D5000E026EA1EC21F0FD0E026E200E016E2D12
:10A8E500EC21F0000E4C6E140E4B6E000E4E6E1EDB
:10A8F5000E4D6E820E4F6E010E506EA1EC30F004BF
:10A905000E016EFF0E026EA1EC21F0000E4C6E449E
:10A915000E4B6E000E4E6E210E4D6EF50E4F6EFFF8
:10A925000E506EA1EC30F0F70E016EFE0E026EA118
:10A93500EC21F0000E4C6E480E4B6E000E4E6E2351
:10A945000E4D6EFB0E4F6EFF0E506EA1EC30F0807B
:10A95500D0660E136E660E146EE60E156E3F0E165D
:10A965006EF1C1F7F0F0C1F6F0EFC1F5F00001F4BA
:10A975006BF4C00FF0F5C010F0F6C011F0F7C0127F
:10A98500F020EC3AF00FC035F010C036F011C037AA
:10A99500F012C038F0000E396E000E3A6E000E3B14
:10A9A5006E420E3C6E82EC38F036C0F8F037C0F9D6
:10A9B500F038C0FAF0F8C067F1F9C068F1FAC0697B
:10A9C500F1820E516E010E526ED70E536EFF0E546C
:10A9D5006E69C1F7F068C1F6F067C1F5F00001F4E2
:10A9E5006BF4C055F0F5C056F0F6C057F0F7C058F7
:10A9F500F0F6EC43F0110E016EFF0E026EA1EC2194
:10AA0500F0FD0E026E200E016E2DEC21F0000E4CB5
:10AA15006E140E4B6E000E4E6E1E0E4D6E820E4F58
:10AA25006E010E506EA1EC30F0F70E016EFE0E02B7
:10AA35006EA1EC21F0000E4C6E480E4B6E000E4ED2
:10AA45006E230E4D6EFD0E4F6EFF0E506EA1EC3057
:10AA5500F05E0E026EFF0E036E24EC24F0820E02F1
:10AA65006E010E036E24EC24F05B0E026EFF0E03E6
:10AA75006E24EC24F01E0E0101DD19D8A493D1003B
:10AA85000EC66F000EC56F410EC55D010EC659D8C5
:10AA9500B01AD0C5C113F0C6C114F0F20EC525D940
:10AAA5006E010EC621DA6EDF500001F46FF4511508
:10AAB5006E166A000E186E000E176ECCEC22F001B1
:10AAC50001C54BC62BE0D7000EC86F000EC76F40FF
:10AAD5000EC75D010EC859D8B01BD0010EC72500A1
:10AAE50001F46F000E0101C8210001F56FF20EF4AB
:10AAF50025D96E010EF521DA6EF20E0101C725E1A9
:10AB05006E010EC821E26EDFCFE7FFC74BC82BDF12
:10AB1500D7F1C1F7F0F0C1F6F0EFC1F5F00001F49F
:10AB25006BF4C00FF0F5C010F0F6C011F0F7C012CD
:10AB3500F0000E136E000E146EC80E156E420E1642
:10AB45006E20EC3AF010C0F8F011C0F9F012C0FA1E
:10AB5500F0F8C0B2F1F9C0B3F1FAC0B4F1000E01DA
:10AB650001E96F000EEA6F000EEB6FB4AF35D0B29E
:10AB7500C101F0B3C102F0B4C103F07DEC21F001D5
:10AB8500C0B2F102C0B3F103C0B4F1B4C1F7F0B380
:10AB9500C1F6F0B2C1F5F00001F46BF4C001F0F5B7
:10ABA500C002F0F6C003F0F7C004F0000E056E0019
:10ABB5000E066EA00E076E400E086E3CEC34F002D9
:10ABC500C0F8F003C0F9F004C0FAF0F8C0E9F1F9F3
:10ABD500C0EAF1FAC0EBF1AED0B4C1F7F0B3C1F6FB
:10ABE500F0B2C1F5F00001F46BF4C001F0F5C0025C
:10ABF500F0F6C003F0F7C004F0000E056E000E0677
:10AC05006EA00E076E400E086E3CEC34F002C0F8E4
:10AC1500F003C0F9F004C0FAF0F8C0E9F1F9C0EAB0
:10AC2500F1FAC0EBF1000E016E340E026E440E0314
:10AC35006EE9C104F0EAC105F0EBC106F0B8EC25F8
:10AC4500F0D8B014D0E9C127F0EAC128F0EBC1294A
:10AC5500F0000E2A6E340E2B6EC40E2C6ED1EC2E27
:10AC6500F027C0E9F128C0EAF129C0EBF1000E0197
:10AC75006EF00E026E430E036EE9C104F0EAC105E3
:10AC8500F0EBC106F0B8EC25F0D8B014D0E9C12737
:10AC9500F0EAC128F0EBC129F0000E2A6EF00E2B68
:10ACA5006EC30E2C6ED1EC2EF027C0E9F128C0EA58
:10ACB500F129C0EBF1000E016E700E026E430E031A
:10ACC5006EE9C104F0EAC105F0EBC106F0B8EC2568
:10ACD500F0D8B014D0E9C127F0EAC128F0EBC129BA
:10ACE500F0000E2A6E700E2B6EC30E2C6ED1EC2E5C
:10ACF500F027C0E9F128C0EAF129C0EBF1E9C1016B
:10AD0500F0EAC102F0EBC103F07DEC21F001C027B0
:10AD1500F002C028F003C029F0000E2A6E6F0E2B3A
:10AD25006E430E2C6ED1EC2EF027C0E9F128C0EA57
:10AD3500F129C0EBF1E9C110F0EAC111F0EBC11244
:10AD4500F056EC29F010C031F3000E0101DA6F0066
:10AD55000ED96F400ED95D010EDA59D8B023D0F265
:10AD65000ED925D96E010EDA21DA6EDF50D8B41668
:10AD7500D0D9C113F0DAC114F0F20ED925D96E017C
:10AD85000EDA21DA6EDF500001F46FF451156E16FC
:10AD95006AFD0E186E200E176ECCEC22F00101D95B
:10ADA5004BDA2BD7D75B0E026EFF0E036E24EC2415
:10ADB500F00101DD2B130E026E880E016E40EC22B0
:10ADC500F0CAEF4AF0000000803F0000204100007B
:10ADD500C84200007A4400401C460050C347002486
:10ADE50074498096184B20BCBE4C286B6E4EF902F8
:10ADF5001550EC78AD60CAF249710000803FCDCCAA
:10AE0500CC3D0AD7233C6F12833A17B7D138ACC56E
:10AE15002737BD37863595BFD63377CC2B325F7054
:10AE25008930FFE6DB2E08E53C1E6042A20D0100DD
:10AE350000000A00000064000000E803000010277D
:10AE45000000A086010040420F008096980000E1B6
:10AE5500F50500CA9A3BFF01990000001388CBFF56
:10AE6500019900000007D08FFF019900000003E859
:10AE75007BFF018700000000007800000000000053
:10AE850000000000000000000000000000000000BD
:10AE950000000000000000000000000000000000AD
:10AEA500000000000000000000000000000000009D
:10AEB500000000000000000000000000E007300C6A
:10AEC5000810642666660240024012481248366C35
:10AED5002424C813300CE007000000000000000027
:10AEE500000000000000000000000000000000005D
:10AEF500E007F00FF81FFC3F9E799E79FE7FFE7FED
:10AF0500EE77EE77DC3B381CF00FE0070000000021
:10AF1500000000000000000000003C3C7E7EFE7F3B
:10AF2500FFFFFFFFFFFFFFFFFFFFFFFFFE7FFE7F2E
:10AF3500FC3FFC3FF81FF00FF00FE007C003800156
:10AF4500000000000000000000000000000080007C
:10AF55008001C001E003E007F00FF81FFC3FFE7F12
:10AF6500FFFFFE7FFC3FF81FF00FE007E003C00185
:10AF750080018000000000000000000000000000CB
:10AF85000000C003E007F00FF00FF00FF00FE0072F
:10AF9500FC3FFE7FFFFFFFFFFFFFFE7F9C39800127
:10AFA5008001C003C003C0030000000000000000D2
:10AFB500000000000000000180018003C007E00FD1
:10AFC500F00FF81FFC3FFE7FFEFFFFFFFFFFFFFFB7
:10AFD500FE7F9C3980018001C003C0030000000092
:10AFE500000000000000000000000000000000005C
:10AFF500000000000000000000000000000000004C
:10B00500000000000000000000000000000000003B
:10B01500000000000000000000000000000000002B
:10B02500000000000000000000000000000000001B
:10B03500000000000000000000000000000000000B
:10B0450000000000000000000000000000000000FB
:10B0550000000000000000000000000000000000EB
:10B0650000000000000000000000000000000000DB
:10B0750000000000000000000000000000000000CB
:10B0850000000000000000000000000000000000BB
:10B0950000000000000000000000000000000000AB
:10B0A500000000000000000000000000000000009B
:10B0B500000000000000000000000030007F007F5D
:10B0C500007800CC00CEF007FC070E0E060C031826
:10B0D5000318031803180318060C0E0EFC07F001DD
:10B0E5000000000000000000000000000000C00794
:10B0F500F01F383818300C600C600C600C601C6058
:10B1050018307838F01FC00F00030003E01FE01F60
:10B115000003000300000000000000000000000024
:10B12500000000000000000000000000000000001A
:10B13500000000000000000000000000000000000A
:10B1450000000000000000000000000000000000FA
:10B1550000000000000000400070007E807FE04796
:10B16500E041204020402040204020402040204019
:10B1750020402078207C207E203E3C1C3E003F0065
:10B185001F000E000000000000000000000000008D
:10B1950080018811DC3BF81F300C18181E781E78CA
:10B1A5001818300CF81FDC3B8811800100000000E6
:10B1B500000000000000000000000000000000008A
:10B1C50000000000000002000E003E00FE00FE012F
:10B1D500FE07FE1FFE7FFE1FFE07FE01FE003E006E
:10B1E5000E0002000000000000000000000000004A
:10B1F5000000000000000000000000400070007C1E
:10B20500007F807FE07FF87FFE7FF87FE07F807F93
:10B21500007F007C0070004000000000000000007E
:10B2250000000000000080018001C003E007B00DB0
:10B235008001800180018001800180018001800101
:10B2450080018001800180018001B00DE007C0030D
:10B2550080018001000000000000701C701C701C43
:10B26500701C701C701C701C701C701C701C701C79
:10B27500701C701C701C00000000701C701C701C81
:10B285000000000000000000000000000000F81FA2
:10B29500FC1FFE18FE18FE18FE18FE18FC18F818FC
:10B2A500F018C018C018C018C018C018C018C018A9
:10B2B500C018C018C018C018C018C0180000000079
:10B2C5000000C01FF01F7810380038007800F0012A
:10B2D500E007F00F301E383C38387838F019E00FA9
:10B2E500800F001E003C00380038183CF81FE007AE
:10B2F5000000000000000000000000000000000049
:10B305000000FE7FFE7FFE7FFE7FFE7F00000000C7
:10B315000000000000000000000000000000000028
:10B32500000000000000000080018001C003E0076C
:10B33500B00D8001800180018001800180018001C4
:10B3450080018001800180018001B00DE007C0030C
:10B35500800180010000F00FF00F00000000800167
:10B365008001C003E007B00D8001800180018001EC
:10B3750080018001800180018001800180018001C0
:10B3850080018001800180018001800100000000B2
:10B395000000800180018001800180018001800121
:10B3A5008001800180018001800180018001800190
:10B3B500800180018001B00DE007C003800180019C
:10B3C5000000000000000000000000000000000078
:10B3D500000000000004000C0018FE7FFE7F00182E
:10B3E500000C000400000000000000000000000048
:10B3F5000000000000000000000000000000000048
:10B405000000000000000000200030001800FE7F52
:10B41500FE7F180030002000000000000000000042
:10B425000000000000000000000000000000000017
:10B4350000000000000000000600060006000600EF
:10B4450006000600060006000600060006000600C7
:10B45500FE7FFE7F000000000000000000000000ED
:10B4650000000000000000000000000000000000D7
:10B475002004300C1818FE7FFE7F1818300C2004AD
:10B4850000000000000000000000000000000000B7
:10B4950000000000000000000000000000000001A6
:10B4A500000180038003C003C007E007E00FF00F31
:10B4B500F01FF81FF81FFC3FFC3FFE7F0000000057
:10B4C5000000000000000000000000000000000077
:10B4D5000000FE7FFC3FFC3FF81FF81FF01FF00F38
:10B4E500E00FE007C007C0038003800300010001EF
:10B4F5000000000000000000000000000000000047
:10B505000000000000000000000000000000000036
:10B515000000000000000000000000000000000026
:10B525000000000000000000000000000000000016
:10B535000000800380038003800380038003800371
:10B545008003800380038003800380038003000061
:10B55500000080038003800300000000000000005D
:10B5650000000000380E380E380E380E380E100464
:10B5750010040000000000000000000000000000B2
:10B5850000000000000000000000000000000000B6
:10B595000000000000000000000080318031C0186C
:10B5A500C018C018C018FC7FFC7F600C6006300610
:10B5B500FE3FFE3F18031803180318038C018C0186
:10B5C5000000000000000000000000030003C01F91
:10B5D500F03F70233803380338037803F003E003A2
:10B5E5008007001F001F003B003B003B003B181B72
:10B5F500F81FE00F0003000300000000000000003A
:10B6050000003CC06660C330C318C318C30CC30632
:10B6150066033C038001C03CC06660C330C318C3E9
:10B6250018C30CC30666033C0000000000000000C0
:10B63500000000000000E003F007380E380E380E59
:10B6450038067007F001F800FCE0CEE1C7E3876338
:10B655000767077E0F3E1E3CFC7FF0F300000000ED
:10B665000000000000000000C001C001C001C001D1
:10B67500C001800080000000000000000000000004
:10B6850000000000000000000000000000000000B5
:10B695000000000000000000000000000018001E6F
:10B6A500000F8003C001E000E000E00070007000C2
:10B6B500700070007000700070007000E000E00025
:10B6C500E000C0018003000F001E0018000000000C
:10B6D5000C003C007800E000C0018003800380037B
:10B6E500000700070007000700070007000700071D
:10B6F500800380038003C001E00078003C000C005B
:10B70500000000000000800380038003981B7C3E3E
:10B71500300C4002E007700E381C200400000000C9
:10B725000000000000000000000000000000000014
:10B735000000000000000000000000000000000004
:10B7450000000000800180018001800180018001EE
:10B75500FE7FFE7F800180018001800180018001E4
:10B7650000000000000000000000000000000000D4
:10B7750000000000000000000000000000000000C4
:10B78500000000000000000000000000C003C0032E
:10B79500C003C003000380038001C0000000000057
:10B7A5000000000000000000000000000000000094
:10B7B500000000000000F81FF81F00000000000056
:10B7C5000000000000000000000000000000000074
:10B7D5000000000000000000000000000000000064
:10B7E5000000000000000000000000000000000054
:10B7F50000000000C003C003C003C0030000000038
:10B80500000000000000000000600030003000185B
:10B815000018000C000C0006000600030003800160
:10B825008001C000C00060006000300030001800DA
:10B8350018000C000C000600000000000000E003EA
:10B84500F007380E1C1C1C1C0E380E380E380E382E
:10B855000E380E380E380E380E381C1C1C1C380ECF
:10B86500F007E003000000000000000000000000F9
:10B8750000000003E003FC038C03800380038003C6
:10B88500800380038003800380038003800380039B
:10B8950080038003FC7FFC7F0000000000000000A7
:10B8A500000000000000F003FC070C0E001C001C4B
:10B8B500001C001C000E000E00078003C001E00004
:10B8C5007000300038001C00FC1FFC1F0000000049
:10B8D50000000000000000000000F003F80F081E43
:10B8E500001C001C001C000C0006E003E007000F14
:10B8F500001E001C001C001C001E080FF807F803A2
:10B905000000000000000000000000000000000E24
:10B91500000F800F800FC00EE00E600E300E180E67
:10B92500180E0C0E060EFE7FFE7F000E000E000E9A
:10B93500000E000E000000000000000000000000E6
:10B945000000F03FF03FF03F3000300030003000A5
:10B955003000F003F00F001E003C003800380038BE
:10B96500003C101EF00FF003000000000000000076
:10B97500000000000000801FE03FF020700038004C
:10B9850038001C009C0FDC1F7C3C3C781C701C7034
:10B995001C70387038387038F01FC0070000000080
:10B9A50000000000000000000000F83FF83FF83FED
:10B9B50000180018000C000C0006000200038001AE
:10B9C5008001C000C00060006000700030003000E1
:10B9D5000000000000000000000000000000C0079B
:10B9E500F00F781E381C381C381C780CF00FE0035B
:10B9F500F00F381F181E1C3C1C381C381C38381C0E
:10BA0500F00FE0070000000000000000000000004B
:10BA15000000C007F01F381C38381C381C701C701B
:10BA25001C703C78787CF077E07300700038003843
:10BA3500001C081EF80FF0030000000000000000C5
:10BA450000000000000000000000000000000000F1
:10BA5500C003C003C003C0030000000000000000D5
:10BA650000000000C003C003C003C00300000000C5
:10BA750000000000000000000000000000000000C1
:10BA850000000000C003C003C003C00300000000A5
:10BA95000000000000000000C003C003C003C00395
:10BAA500000380038001C0000000000000000000CA
:10BAB500000000000000000000400070003C000F86
:10BAC500C003F0003C003C00F000C003000F003C48
:10BAD50000700040000000000000000000000000B1
:10BAE5000000000000000000000000000000000051
:10BAF5000000FE7FFE7F000000000000FE7FFE7F4D
:10BB05000000000000000000000000000000000030
:10BB15000000000000000000000000000000000020
:10BB250002000E003C00F000C003000F003C003C8A
:10BB3500000FC003F0003C000E00020000000000F2
:10BB450000000000000000000000F807FC1F0C3C8E
:10BB55000C3800380038001C001E000F80078003D9
:10BB6500C001C001C00100000000C001C001C0014A
:10BB75000000000000000000000000000000C00FF1
:10BB8500E01F703818301C3E0C318E31C630C6307F
:10BB9500C638C638C63CC6348EF78CF31C00380848
:10BBA500F00FC007000000000000000000000000CA
:10BBB5000000000000000000C001C003E0036007B2
:10BBC50060077006300E380E381C181CFC3FFC3F11
:10BBD5000E380E700E7007E0000000000000000037
:10BBE500000000000000000000000000FC07FC0F42
:10BBF5001C1E1C1C1C1C1C0EFC07FC071C1E1C3CD4
:10BC05001C381C381C381C3CFC1FFC0700000000BD
:10BC1500000000000000000000000000000000001F
:10BC2500C01FF03F78303C001C000E000E000E00D7
:10BC35000E000E000E001C003C007820F03FC01FD7
:10BC450000000000000000000000000000000000EF
:10BC550000000000FC07FC0F1C3C1C381C781C7005
:10BC65001C701C701C701C701C701C381C381C1E31
:10BC7500FC0FFC03000000000000000000000000B5
:10BC85000000000000000000F83FF83F38003800D1
:10BC9500380038003800F81FF81F38003800380021
:10BCA50038003800F87FF87F000000000000000031
:10BCB500000000000000000000000000F87FF87F91
:10BCC50038003800380038003800F83FF83F3800B1
:10BCD500380038003800380038003800000000000F
:10BCE500000000000000000000000000000000004F
:10BCF500C01FF03F78303C001C000E000E000E0007
:10BD05000E3F0E3F0E381C383C387838F03FC01FC8
:10BD1500000000000000000000000000000000001E
:10BD2500000000001C381C381C381C381C381C3816
:10BD35001C38FC3FFC3F1C381C381C381C381C3890
:10BD45001C381C3800000000000000000000000046
:10BD55000000000000000000FC1FFC1FC001C00126
:10BD6500C001C001C001C001C001C001C001C001C6
:10BD7500C001C001FC1FFC1F000000000000000006
:10BD8500000000000000000000000000F80FF80FA0
:10BD9500000E000E000E000E000E000E000E000E2E
:10BDA500000E000E000E0407FC03FC01000000005D
:10BDB500000000000000000000000000000000007E
:10BDC5001C781C3C1C1E1C0F1C079C03DC01FC0082
:10BDD500DC01DC039C071C0F1C1E1C3C1C781CF89A
:10BDE500000000000000000000000000000000004E
:10BDF50000000000380038003800380038003800EE
:10BE0500380038003800380038003800380038006D
:10BE1500F83FF83F000000000000000000000000AF
:10BE250000000000000000000E381E3C1E3C1E3CB9
:10BE3500363636363636663266336633C631C63101
:10BE4500C631063006300630000000000000000054
:10BE55000000000000000000000000001C301C3045
:10BE65003C307C307C30FC30EC31CC31CC338C3701
:10BE75000C3F0C3E0C3E0C3C0C380C38000000000E
:10BE850000000000000000000000000000000000AD
:10BE9500E007F00F381C1C381C380E700E700E7041
:10BEA5000E700E700E701C381C38381CF00FE00731
:10BEB500000000000000000000000000000000007D
:10BEC50000000000F81FF83F387838703870387077
:10BED5003878383CF81FF807380038003800380043
:10BEE50038003800000000000000000000000000DD
:10BEF5000000000000000000E007F00F381C1C38AF
:10BF05001C380E700E700E700E700E700E701C3890
:10BF15001C38381CF00FE007001E007800F00040C8
:10BF2500000000000000000000000000FC07FC0FFE
:10BF35001C1E1C1C1C1C1C1C1C0EFC07FC039C074B
:10BF45001C071C0F1C1E1C3C1C381C780000000024
:10BF550000000000000000000000000000000000DC
:10BF6500E00FF81F3C181C001C003C00F800F0070F
:10BF7500C01F003E0038003800380C1CFC1FF007BD
:10BF850000000000000000000000000000000000AC
:10BF950000000000FF7FFF7FC001C001C001C0019C
:10BFA500C001C001C001C001C001C001C001C00184
:10BFB500C001C001000000000000000000000000FA
:10BFC50000000000000000001C701C701C701C703C
:10BFD5001C701C701C701C701C701C701C701C70FC
:10BFE5003C783838F01FE00F00000000000000002A
:10BFF50000000000000000000000000007E00E70D7
:10C005000E701C701C383C383838381C701C700C8D
:10C01500E00EE00EE007C007C00780030000000047
:10C02500000000000000000000000000000000000B
:10C0350003C003C007C08661C663C663C663C66323
:10C045004E766C366C366C362C3E3C3C3C1C3C1CAF
:10C0550000000000000000000000000000000000DB
:10C06500000000001EE03C707838781CF00EE007F8
:10C07500C003C003C007E007600F301E183C1C3822
:10C085000E7807F00000000000000000000000002E
:10C09500000000000000000007E00E701C301C18B6
:10C0A500381C780E7007E003E003C001C001C00131
:10C0B500C001C001C001C001000000000000000077
:10C0C500000000000000000000000000FC3FFC3FF5
:10C0D5000038001C000E000780038001C000E0004E
:10C0E500700038001C000E00FE3FFE3F00000000FF
:10C0F5000000000000000000C03FC03FC001C001BB
:10C10500C001C001C001C001C001C001C001C00122
:10C11500C001C001C001C001C001C001C001C00112
:10C12500C001C001C03FC03F0000000006000C0078
:10C135000C00180018003000300060006000C000DE
:10C14500C000800180010003000300060006000C0A
:10C15500000C0018001800300030006000000000DE
:10C16500FC03FC03800380038003800380038003BA
:10C1750080038003800380038003800380038003A2
:10C18500800380038003800380038003FC03FC039A
:10C195000000000000000001000180038003C003CF
:10C1A500C006E006600C300C3018181818180C3052
:10C1B5000C300660000000000000000000000000D8
:10C1C500000000000000000000000000000000006A
:10C1D500000000000000000000000000000000005A
:10C1E500000000000000000000000000000000004A
:10C1F500FFFFFFFF000000000000C00180030007F3
:10C205000000000000000000000000000000000029
:10C215000000000000000000000000000000000019
:10C225000000000000000000000000000000000009
:10C23500000000000000000000000000E007F80F0B
:10C24500181E001C001CE01FF01F381C1C1C1C1CA9
:10C255001C1C3C1EF87BF07800000000000000006C
:10C26500000000001C001C001C001C001C001C0021
:10C275009C07DC1F7C1C3C381C381C381C381C38BF
:10C285001C381C381C1C3C1EFC0FCC070000000091
:10C295000000000000000000000000000000000099
:10C2A50000000000C01FF03F782038001C001C0073
:10C2B5001C001C001C003C003800F820F03FC01F8B
:10C2C5000000000000000000000000000070007089
:10C2D5000070007000700070C073F07F787C38705B
:10C2E5001C701C701C701C701C701C703C78387C99
:10C2F500F077E0730000000000000000000000007F
:10C30500000000000000000000000000C007F00F62
:10C31500781C38381C381C38FC3FFC3F1C001C00BE
:10C3250038007820F03FC01F00000000000000002A
:10C335000000000000FF80FFC003C001C001C00174
:10C34500FC7FFC7FC001C001C001C001C001C0016C
:10C35500C001C001C001C001C001C0010000000052
:10C3650000000000000000000000000000000000C8
:10C3750000000000C073F07F787C38701C701C7062
:10C385001C701C701C701C703C78387CF077E07356
:10C3950000700038183CF81FF00700001C001C0056
:10C3A5001C001C001C001C001C0FDC1F7C3C3C38C6
:10C3B5001C381C381C381C381C381C381C381C38D8
:10C3C5001C381C38000000000000000000000000C0
:10C3D500800380038003000000000000FC03FC03D1
:10C3E5008003800380038003800380038003800330
:10C3F500800380038003800300000000000000002C
:10C4050000000000000E000E000E000000000000FD
:10C41500F80FF80F000E000E000E000E000E000EB5
:10C42500000E000E000E000E000E000E000E000E97
:10C435000407FC07F8010000380038003800380010
:10C4450038003800383C381E380E380FB807B803A6
:10C45500F803B803B807380F380E381E383C38785B
:10C46500000000000000000000000000F807F807C9
:10C47500000700070007000700070007000700077F
:10C48500000700070007000700070007000700076F
:10C495000007000700000000000000000000000089
:10C4A500000000000000000000000000CE31EE7921
:10C4B500FE7F9E779E738E738E738E738E738E73CF
:10C4C5008E738E738E738E73000000000000000063
:10C4D5000000000000000000000000000000000057
:10C4E5001C0FDC1F7C3C3C381C381C381C381C38A5
:10C4F5001C381C381C381C381C381C38000000003F
:10C505000000000000000000000000000000000026
:10C5150000000000E003F80F3C1E1C1C0E380E380E
:10C525000E380E380E380E381C1C3C1EF80FE00372
:10C5350000000000000000000000000000000000F6
:10C5450000000000000000009C07DC1F7C1C3C383C
:10C555001C381C381C381C381C381C381C1C3C1E4C
:10C56500FC0F9C071C001C001C001C001C0000008C
:10C57500000000000000000000000000E039F83F66
:10C585003C3E1C380E380E380E380E380E380E3834
:10C595001E3C1C3EF83BF0380038003800380038A7
:10C5A500003800000000000000000000000000004E
:10C5B500703E703FF031F030700070007000700018
:10C5C50070007000700070007000700000000000C6
:10C5D5000000000000000000000000000000000056
:10C5E50000000000E00FF01F781038003800F80157
:10C5F500F007801F003C00380038183CF81FF00792
:10C605000000000000000000000000000000000025
:10C6150000000000E000E000FC3FFC3FE000E0001F
:10C62500E000E000E000E000E000E000E000E00104
:10C63500C03F803F00000000000000000000000037
:10C645000000000000000000000000001C381C383D
:10C655001C381C381C381C381C381C381C381C3835
:10C665001C3C3C3EF83BF038000000000000000098
:10C6750000000000000000000000000000000000B5
:10C685001E701C381C383C383818381C701C700C4F
:10C69500E00EE00EE006C007C007800300000000C2
:10C6A5000000000000000000000000000000000085
:10C6B5000000000003C087C38743C663C6634662A4
:10C6C5006E666E266C362C363C3C3C3C3C1C181C7D
:10C6D5000000000000000000000000000000000055
:10C6E50000000000000000001E303C18780C700EA1
:10C6F500F006E003C003C003E007700F300E381EDC
:10C705001C3C0E7800000000000000000000000046
:10C715000000000000000000000000001E701C303A
:10C725001C383818381C781C700EF00EE007E0072E
:10C73500C003C003C0018001C001C000E0007C004F
:10C745003C000000000000000000000000000000A8
:10C75500FC3FFC3F0038001C000E00078003C001B1
:10C76500E000700038001C00FC3FFC3F00000000AA
:10C775000000000000000000001F801FC003C00172
:10C78500C001C0018003800380038003C001F8005D
:10C79500F800C0018003800380038003C001C0014D
:10C7A500C001C003801F001F000000008001800140
:10C7B500800180018001800180018001800180016C
:10C7C500800180018001800180018001800180015C
:10C7D500800180018001800180018001000000004E
:10C7E5007C00FC00E001C001C001C001E000E000E8
:10C7F500E000E000C001800F800FC001E000E00014
:10C80500E000E000C001C001C001E001FC007C00C7
:10C815000000000000000000000000000000000013
:10C82500000000000000000000007860FC63C63FC7
:10C83500061E0000000000000000000000000000CF
:10C8450000000000000000000000000000000000E3
:10C85500F80F08080808080808080808080808085C
:10C865000808080808080808080808080808F80F4C
:10C8750000000000000000000000000000000000B3
:10C8850000000000C01FF03F78303C001C000E0087
:10C895000E000E000E000E000E001C003C0078205D
:10C8A500F03FC01F00020007000C000C80070000CD
:10C8B5000000000030063006000000001C381C385F
:10C8C5001C381C381C381C381C381C381C381C38C3
:10C8D5001C3C3C3EF83BF038000000000000000026
:10C8E50000000000000C00060003800100000000AD
:10C8F500C007F00F781C38381C381C38FC3FFC3F4B
:10C905001C001C0038007820F03FC01F000000000C
:10C915000000000000000000C00160033006180C94
:10C9250000000000E007F80F181E001C001CE01FA7
:10C93500F01F381C1C1C1C1C1C1C3C1EF87BF078B2
:10C9450000000000000000000000000000000000E2
:10C95500600C600C00000000E007F80F181E001CBA
:10C96500001CE01FF01F381C1C1C1C1C1C1C3C1E42
:10C97500F87BF078000000000000000000000000D7
:10C9850030006000C000800100000000E007F80FE3
:10C99500181E001C001CE01FF01F381C1C1C1C1C52
:10C9A5001C1C3C1EF87BF078000000000000000015
:10C9B5000000C001200220022002C001000000008A
:10C9C500E007F80F181E001C001CE01FF01F381CA4
:10C9D5001C1C1C1C1C1C3C1EF87BF0780000000075
:10C9E5000000000000000000000000000000000042
:10C9F50000000000C01FF03F782038001C001C001C
:10CA05001C001C001C003C003800F820F03FC01F33
:10CA15000001800300060006C0030000C00160039A
:10CA25003006180C00000000C007F00F781C3838DD
:10CA35001C381C38FC3FFC3F1C001C0038007820CB
:10CA4500F03FC01F000000000000000000000000D3
:10CA550000000000600C600C00000000C007F00F33
:10CA6500781C38381C381C38FC3FFC3F1C001C0067
:10CA750038007820F03FC01F0000000000000000D3
:10CA85000000000030006000C000800100000000D0
:10CA9500C007F00F781C38381C381C38FC3FFC3FA9
:10CAA5001C001C0038007820F03FC01F000000006B
:10CAB5000000000000000000000000003006300605
:10CAC50000000000FC03FC03800380038003800357
:10CAD5008003800380038003800380038003800339
:10CAE5000000000000000000000000008003C006F8
:10CAF500600C301800000000FC03FC038003800379
:10CB05008003800380038003800380038003800308
:10CB1500800380030000000000000000000000000A
:10CB25006000C0008001000300000000FC03FC035E
:10CB350080038003800380038003800380038003D8
:10CB450080038003800380030000000000000000D4
:10CB55000000300C300C000000000000C001C003D4
:10CB6500E003600760077006300E380E381C181C8D
:10CB7500FC3FFC3F0E380E700E7007E00000000011
:10CB850000000000000080034004400440048003CE
:10CB95008003C007C007E006600E600E700C301CF5
:10CBA500381C3838FC3FFC3F1C700E700E7007E0D7
:10CBB50000000000000000000000000E00078003D8
:10CBC50000000000F83FF83F380038003800380012
:10CBD5003800F81FF81F38003800380038003800D2
:10CBE500F87FF87F00000000000000000000000052
:10CBF500000000000000000000000000F83CFC7F81
:10CC0500806780E380E3F0FFFCFF9C038E038E03C7
:10CC15008E039E87FCFF787C00000000000000006A
:10CC2500000000000000000000000000803FC03F41
:10CC3500C007E007600760077007303F383F1807F7
:10CC45001C07FC07FC070607067F037F00000000A2
:10CC55000000000000000000C00160033006180C51
:10CC650000000000E003F80F3C1E1C1C0E380E38B7
:10CC75000E380E380E380E381C1C3C1EF80FE0031B
:10CC8500000000000000000000000000000000009F
:10CC95003006300600000000E003F80F3C1E1C1CA7
:10CCA5000E380E380E380E380E380E381C1C3C1E49
:10CCB500F80FE00300000000000000000000000085
:10CCC50030006000C000800100000000E003F80FA4
:10CCD5003C1E1C1C0E380E380E380E380E380E3819
:10CCE5001C1C3C1EF80FE0030000000000000000C3
:10CCF50000000000C00160033006180C00000000B1
:10CD05001C381C381C381C381C381C381C381C387E
:10CD15001C381C381C3C3C3EF83BF0380000000039
:10CD2500000000000000000030006000C00080012D
:10CD3500000000001C381C381C381C381C381C38F6
:10CD45001C381C381C381C381C3C3C3EF83BF03861
:10CD550000000000000000000000000000000000CE
:10CD650030063006000000001E701C301C383818D4
:10CD7500381C781C700EF00EE007E007C003C003F6
:10CD8500C0018001C001C000E0007C003C00300C07
:10CD9500300C000000000000E007F00F381C1C38C4
:10CDA5001C380E700E700E700E700E700E701C38E2
:10CDB5001C38381CF00FE0070000000000000000E0
:10CDC5000000601860180000000000001C701C7056
:10CDD5001C701C701C701C701C701C701C701C70EE
:10CDE5001C701C703C783838F01FE00F0000000004
:10CDF500000000000000000000000000000000002E
:10CE050000000000E033F81F3C1E1C1E0E3B0E39CF
:10CE15008E39CE386E386E383C1C3C1EFC0FE6034E
:10CE25000000000000000000000000000000003EBF
:10CE3500803F8003C001C001C001C001C001F00FE7
:10CE4500F00FC001C001C001C001E0007000F83F53
:10CE5500F83FF83F0000000000000000000000005F
:10CE65000000000000000000E067F03F381C1C3C9B
:10CE75001C3C0E760E738E718E71CE706E703C38C2
:10CE85003C38381CFC0FE6070000000000000000DD
:10CE9500000000000000000000000000000000008D
:10CEA50004200E701C38381C700EE007C003C00348
:10CEB500E007700E381C1C380E70042000000000BE
:10CEC5000000000000000000003F803FC001C001DD
:10CED500C001C001F81FF81FC001C001C001C00199
:10CEE500C001C001C001C001C001C001C001C00135
:10CEF500C001C001C001FE007E0000000006000365
:10CF05008001C00000000000E007F80F181E001C9B
:10CF1500001CE01FF01F381C1C1C1C1C1C1C3C1E8C
:10CF2500F87BF07800000000000000000000000021
:10CF3500000600038001C00000000000FC03FC03A4
:10CF450080038003800380038003800380038003C4
:10CF550080038003800380030000000000000000C0
:10CF650000000000000600038001C0000000000072
:10CF7500E003F80F3C1E1C1C0E380E380E380E3818
:10CF85000E380E381C1C3C1EF80FE0030000000094
:10CF95000000000000000000000600038001C00042
:10CFA500000000001C381C381C381C381C381C3884
:10CFB5001C381C381C381C381C3C3C3EF83BF038EF
:10CFC5000000000000000000000000000000E00C70
:10CFD500F00F3007000000001C0FDC1F7C3C3C38C4
:10CFE5001C381C381C381C381C381C381C381C389C
:10CFF5001C381C3800000000000000000000E00C98
:10D00500F00F3007000000001C301C303C307C3035
:10D015007C30FC30EC31CC31CC338C370C3F0C3EC2
:10D025000C3E0C3C0C380C380000000000000000E1
:10D03500000000000000E003F0071006E007F0071D
:10D04500380618061807F81FF01C0000000000003D
:10D0550000000000000000000000000000000000CB
:10D0650000000000000000000000E007F00F381C81
:10D075001818181818181818381CF00FE0070000B1
:10D08500000000000000000000000000000000009B
:10D09500000000000000000000000000000000008B
:10D0A50000000000000000008003800380030000F2
:10D0B5000000800380038003C001E001F0007800D8
:10D0C50038001C001C001C303C30F83FE01F0000FD
:10D0D5000000E0031004E80924122412E4112411CD
:10D0E5002411280B1004E0030000000000000000DC
:10D0F500000000000000000000000000000000002B
:10D10500000000000000000000000000000000001A
:10D115000000000000000000FE7FFE7F0060006050
:10D12500006000600000000000000000000000003A
:10D13500000000000000000000001F0C1F061C0678
:10D145001C031C039C019C01DC00DC007C3C30FEC4
:10D1550030E018E018700C380C0C060606FE03FECD
:10D1650000000000000000000000000000001F1883
:10D175001F0C1C0C1C061C061C031C039C019C019B
:10D18500DC38603C603A3039B039D838D8FF0C38D3
:10D195000C38063800000000000000000000000008
:10D1A500000000000000000000000000C001C001F8
:10D1B500C00100000000C001C001C001C001C001E4
:10D1C500C001C001C001C001C001C001C001C00152
:10D1D500C001000000000000000000000000000089
:10D1E50000004010E038701C380E1C070C038E033D
:10D1F5001C07380E701CE0384010000000000000CD
:10D205000000000000000000000000000000000019
:10D2150000000000000008019C033807700EE01CA8
:10D22500C039C018E01C700E38079C0308010000C7
:10D2350000000000000000000000E71CE71CE71CE0
:10D2450000000000E71CE71CE71C00000000E71CCD
:10D25500E71CE71C000000000000E71CE71CE71CBA
:10D2650000000000E71CE71CE71C0000000038E791
:10D2750038E738E7E71CE71CFFFF38E738E7E71C26
:10D28500E71CFFFF38E738E7E71CE71CE71C38E732
:10D2950038E7FFFFE71CE71C38E738E7FFFFE71C27
:10D2A500E71CFFFFFFFFFFFFE71CE71CFFFFFFFF7A
:10D2B500FFFFE71CE71CFFFFFFFFFFFFE71CE71C65
:10D2C500E71CFFFFFFFFFFFFE71CE71CFFFFFFFF5A
:10D2D500FFFFE71CE71C80018001800180018001C0
:10D2E5008001800180018001800180018001800131
:10D2F5008001800180018001800180018001800121
:10D305008001800180018001800180018001800110
:10D315008001800180018001800180018001800100
:10D325008001FF01FF0180018001800180018001F2
:10D33500800180018001800180018001800100075A
:10D345008003C00100000000C001C003E0036007C6
:10D3550060077006300E380E381C181CFC3FFC3F69
:10D365000E380E700E7007E000000000000000008F
:10D375000000E0037007380E00000000C001C00384
:10D38500E003600760077006300E380E381C181C65
:10D39500FC3FFC3F0E380E700E7007E000000000E9
:10D3A500000000000000E000C00180030000000054
:10D3B500C001C003E003600760077006300E380E39
:10D3C500381C181CFC3FFC3F0E380E700E7007E031
:10D3D5000000000000000000000000000000E00F59
:10D3E500F01F38381C708C6FEEEF66C836C036C03B
:10D3F50036C036C036C066C8EEEF8C671C7038384C
:10D40500F01FE00F000000000000000000006006B3
:10D4150060066006600660066006600660066006D7
:10D4250060067F067F06000600067F067F0660060B
:10D4350060066006600660066006600660066006B7
:10D4450060066006600660066006600660066006A7
:10D455006006600660066006600660066006600697
:10D465006006600660066006600660066006600687
:10D475006006600660060000000000000000000075
:10D4850000000000000000000000FF07FF07000685
:10D4950000067F067F066006600660066006600679
:10D4A5006006600660066006600660066006600647
:10D4B50060066006600660066006600660067F0618
:10D4C5007F0600060006FF07FF07000000000000BA
:10D4D5000000000000000000000000000000000047
:10D4E500000080018001C00FF00FB809B8019C0150
:10D4F5009C019C019C019C019C019C01B801F809BF
:10D50500F00FE0078001800100000000000000002E
:10D515000000000000000EE01C6038303830701844
:10D52500E00CE00CC0078003F83FF83F8003800360
:10D535008003F83FF83F800380038003000000006C
:10D5450000000000000000000000000000000000D6
:10D555000000000000000000000000000000FF01C6
:10D56500FF0180018001800180018001800180012F
:10D57500800180018001800180018001800180019E
:10D58500800180018001800180018001800180018E
:10D59500800180FF80FF0000000000000000000007
:10D5A50000000000000000000000000000008001F5
:10D5B500800180018001800180018001800180015E
:10D5C500800180018001FFFFFFFF000000000000D7
:10D5D5000000000000000000000000000000000046
:10D5E5000000000000000000000000000000000036
:10D5F50000000000000000000000FFFFFFFF8001A9
:10D60500800180018001800180018001800180010D
:10D6150080018001800180018001800180018001FD
:10D62500800180018001800180018001800180FFEF
:10D6350080FF8001800180018001800180018001DF
:10D645008001800180018001800100000000000050
:10D6550000000000000000000000000000000000C5
:10D665000000FFFFFFFF00000000000000000000B9
:10D675000000000000000000000000000000800124
:10D68500800180018001800180018001800180018D
:10D69500800180018001FFFFFFFF80018001800183
:10D6A500800180018001800180018001800180016D
:10D6B500800100000000E00CF00F300700000000C2
:10D6C500E007F80F181E001C001CE01FF01F381C97
:10D6D5001C1C1C1C1C1C3C1EF87BF0780000000068
:10D6E500000000000000E00CF00F30070000000013
:10D6F500C001C003E003600760077006300E380EF6
:10D70500381C181CFC3FFC3F0E380E700E7007E0ED
:10D7150000000000000000000000600660066006D2
:10D72500600660066006600660066006600660FECC
:10D7350060FE60006000E0FFE0FF00000000000008
:10D7450000000000000000000000000000000000D4
:10D7550000000000000000000000000000000000C4
:10D765000000E0FFE0FF6000600060FE60FE600614
:10D775006006600660066006600660066006600674
:10D785006006600660066006600660066006600664
:10D795006006600660067FFE7FFE00000000FFFF5A
:10D7A500FFFF000000000000000000000000000076
:10D7B5000000000000000000000000000000000064
:10D7C50000000000000000000000FFFFFFFF000058
:10D7D50000007FFE7FFE600660066006600660064C
:10D7E5006006600660066006600660066006600604
:10D7F500600660066006600660066006600660FEFC
:10D8050060FE6000600060FE60FE60066006600607
:10D815006006600660066006600660066006000039
:10D8250000000000000000000000000000000000F3
:10D835000000FFFFFFFF00000000FFFFFFFF0000EB
:10D8450000000000000000000000000000000000D3
:10D8550000006006600660066006600660066006F9
:10D865006006600660067FFE7FFE000000007FFE0A
:10D875007FFE60066006600660066006600660065C
:10D885006006600660060000000000000000000061
:10D8950000000420CC33F81F300C1818181818187D
:10D8A5001818300CF81FCC330420000000000000CD
:10D8B5000000000000000000000000001E03FE0341
:10D8C500F001F0031807000EE00FF81F3C1E1C3C8A
:10D8D5000E380E380E380E380E380E381C1C3C1E0D
:10D8E500F80FE00300000000000000000000000049
:10D8F5000000000000000000FC07FC0F1C3C1C3869
:10D905001C781C701C70FF70FF701C701C701C381C
:10D915001C381C1EFC0FFC0300000000000000006A
:10D925000000C007E00E701C00000000F83FF83F43
:10D9350038003800380038003800F81FF81F380064
:10D945003800380038003800F87FF87F0000000004
:10D9550000000000000060186018000000000000D2
:10D96500F83FF83F38003800380038003800F81F15
:10D97500F81F38003800380038003800F87FF87F85
:10D9850000000000000000000000C0018003000747
:10D9950000000000F83FF83F380038003800380034
:10D9A5003800F81FF81F38003800380038003800F4
:10D9B500F87FF87F00000000000000000000000074
:10D9C500000000000000000000000000FC03FC0354
:10D9D500800380038003800380038003800380032A
:10D9E5008003800380038003000000000000000026
:10D9F500000000078003C00100000000FC1FFC1FA1
:10DA0500C001C001C001C001C001C001C001C00109
:10DA1500C001C001C001C001FC1FFC1F00000000C7
:10DA2500000000000000E0037007380E0000000051
:10DA3500FC1FFC1FC001C001C001C001C001C00125
:10DA4500C001C001C001C001C001C001FC1FFC1F15
:10DA550000000000000000000000300C300C000049
:10DA650000000000FC1FFC1FC001C001C001C00177
:10DA7500C001C001C001C001C001C001C001C00199
:10DA8500FC1FFC1F000000000000000000008001DA
:10DA95008001800180018001800180018001800179
:10DAA500800180018001FF01FF01000000000000EE
:10DAB5000000000000000000000000000000000061
:10DAC5000000000000000000000000000000000051
:10DAD5000000000000000000000080FF80FF8001C2
:10DAE5008001800180018001800180018001800129
:10DAF500800180018001FFFFFFFFFFFFFFFFFFFFA8
:10DB0500FFFFFFFFFFFFFFFFFFFFFFFFFFFFFFFF20
:10DB1500FFFFFFFFFFFFFFFFFFFFFFFFFFFFFFFF10
:10DB2500FFFFFFFFFFFFFFFFFFFF000000000000FA
:10DB350000000000000000000000000000000000E0
:10DB450000000000FFFFFFFFFFFFFFFFFFFFFFFFDC
:10DB5500FFFFFFFFFFFFFFFFFFFFFFFFFFFF0000CE
:10DB650080018001800180018001800180018001A8
:10DB7500800100000000000000000000800180011D
:10DB85008001800180018001800180018001800188
:10DB95000000E000C001800300000000FC1FFC1F26
:10DBA500C001C001C001C001C001C001C001C00168
:10DBB500C001C001C001C001FC1FFC1F0000000026
:10DBC500000000000000FFFFFFFFFFFFFFFFFFFF5A
:10DBD500FFFFFFFFFFFFFFFFFFFFFFFFFFFFFFFF50
:10DBE5000000000000000000000000000000000030
:10DBF5000000000000000000000000078003C001D5
:10DC050000000000E007F00F381C1C381C380E70AF
:10DC15000E700E700E700E700E701C381C38381C8D
:10DC2500F00FE00700000000000000000000000009
:10DC3500F003F8073C0E1C0E1C0E1C061C079C036B
:10DC45009C039C039C071C0F1C1E1C3C1C781C7011
:10DC55001C709C709C3F1C1F000000000000000011
:10DC65000000E0037007380E00000000E007F00F29
:10DC7500381C1C381C380E700E700E700E700E702D
:10DC85000E701C381C38381CF00FE007000000002F
:10DC9500000000000000E000C0018003000000005B
:10DCA500E007F00F381C1C381C380E700E700E7013
:10DCB5000E700E700E701C381C38381CF00FE00703
:10DCC5000000000000000000000000000000E00C63
:10DCD500F00F300700000000E003F80F3C1E1C1C8D
:10DCE5000E380E380E380E380E380E381C1C3C1EF9
:10DCF500F80FE00300000000000000000000E00C49
:10DD0500F00F300700000000E007F00F381C1C384A
:10DD15001C380E700E700E700E700E700E701C3862
:10DD25001C38381CF00FE007000000000000000060
:10DD350000000000000000000000000000000000DE
:10DD45001C381C381C381C381C381C381C381C382E
:10DD55001C381C383C3C7C3EFC3BDC7B1C001C001E
:10DD65001C001C001C0000001C001C001C001C00EA
:10DD75001C001C009C07DC1F7C1C3C381C381C3814
:10DD85001C381C381C381C381C1C3C1EFC0F9C07FE
:10DD95001C001C001C001C001C00000000000000F2
:10DDA50000000000380038003800F81FF83F3878C8
:10DDB5003870387038703878383CF81FF8073800F4
:10DDC50038003800000000000000000000000007D7
:10DDD5008003C001000000001C701C701C701C70CA
:10DDE5001C701C701C701C701C701C701C701C70CE
:10DDF5003C783838F01FE00F0000000000000000FC
:10DE05000000E0037007380E000000001C701C7055
:10DE15001C701C701C701C701C701C701C701C709D
:10DE25001C701C703C783838F01FE00F00000000B3
:10DE3500000000000000E000C001800300000000B9
:10DE45001C701C701C701C701C701C701C701C706D
:10DE55001C701C701C701C703C783838F01FE00F6B
:10DE650000000000000000000000000000060003A4
:10DE75008001C000000000001E701C301C383818DE
:10DE8500381C781C700EF00EE007E007C003C003D5
:10DE9500C0018001C001C000E0007C003C0000071B
:10DEA5008003C0010000000007E00E701C301C1844
:10DEB500381C780E7007E003E003C001C001C00103
:10DEC500C001C001C001C001000000000000000049
:10DED5000000FFFFFFFF0000000000000000000041
:10DEE500000000000000000000000000000000002D
:10DEF500000000000000000000000000000000001D
:10DF05000000000000008003C001E00000000000E8
:10DF150000000000000000000000000000000000FC
:10DF250000000000000000000000000000000000EC
:10DF350000000000000000000000000000000000DC
:10DF450000000000000000000000000000000000CC
:10DF55000000F81FF81F000000000000000000008E
:10DF650000000000000000000000000000000000AC
:10DF7500000000000000000000000000800180019A
:10DF850080018001FE7FFE7F80018001800180018C
:10DF950000000000FE7FFE7F000000000000000082
:10DFA500000000000000000000000000000000006C
:10DFB500000000000000000000000000000000005C
:10DFC500000000000000000000000000FFFFFFFF50
:10DFD50000000000FFFF000000007EE0FE70E0385A
:10DFE500E0383C1C7C1CE00EE007FE07BE3BC03D54
:10DFF500C03BE039F039F038F8FF38381C380E38B6
:10E005000000000000000000000000000000F81FF4
:10E01500FC1FFE18FE18FE18FE18FE18FC18F8184E
:10E02500F018C018C018C018C018C018C018C018FB
:10E03500C018C018C018C018C018C01800000000CB
:10E045000000C01FF01F7810380038007800F0017C
:10E05500E007F00F301E383C38387838F019E00FFB
:10E06500800F001E003C00380038183CF81FE00700
:10E07500000000000000000000000000000000009B
:10E08500C001C001C001000000000000FE3FFE3FCE
:10E09500000000000000C001C001C0010000000038
:10E0A500000000000000000000000000000000006B
:10E0B500000000000000000000000000000000005B
:10E0C500000000000000000000000000000000004B
:10E0D5000001800300060006C00300000000E00008
:10E0E500100110011001E000000000000000000018
:10E0F500000000000000000000000000000000001B
:10E105000000000000000000000000000000300CCE
:10E11500300C0000000000000000000000000000BE
:10E1250000000000000000000000000000000000EA
:10E1350000000000000000000000000000000000DA
:10E1450000000000000000000000000000000000CA
:10E15500000000000000000000000000C001C00138
:10E16500C0010000000000000000000000000000E9
:10E1750000000000000000000000E003E003800351
:10E1850080038003800380038003800380030000F5
:10E19500000000000000000000000000000000007A
:10E1A5000000000000000000000000000000E00F7B
:10E1B500F01F101C001CC007C00F001C001CF01F26
:10E1C500F007000000000000000000000000000053
:10E1D500000000000000000000000000000000003A
:10E1E5000000E007F01F101C001C000E8007C00196
:10E1F5007000F01FF01F000000000000000000008C
:10E205000000000000000000000000000000000009
:10E2150000000000000000000000000000000000F9
:10E22500FE7FFE7FFE7FFE7FFE7FFE7FFE7FFE7F01
:10E23500FE7FFE7FFE7FFE7FFE7FFE7F00000000EB
:10E2450000000000000000000000000000000000C9
:10E2550000000000000000000000000000000000B9
:10E2650000000000000000000000000000000000A9
:10E275000000000000000000000000000000000099
:10E285000000000000000000000000003C42A581E5
:10E29500BD423C000000000000003C7EDBFFDB428D
:10E2A5003C0000000066FFFFFFFF7E7E3C3C18003F
:10E2B50000000010183C7EFF7E3C38101000000066
:10E2C50000183C3C7EFFFF6E181818000000001077
:10E2D50018387CFEFFFF6E181800000000000000D3
:10E2E5000000000000000000000000000000000029
:10E2F5000000000000000000000000000000000019
:10E305000000000000000000000000000000000008
:10E31500000000000060D0A03C22414141221C00C9
:10E325000000001C22414141221C083E080000005B
:10E335000000000000000000000000000000004098
:10E3450070584848484848783E0F070000000008C4
:10E355007E46C3467E080000000000000001073F1E
:10E36500FF3F0F070100000000000080E0FCFFFCFC
:10E37500F0E080000000001038541010101010104C
:10E3850054381000002424242424242400242400A8
:10E395000000007E4F4F4F4E4848484848484800C7
:10E3A500007804041C34444C386040443C000000B0
:10E3B5000000007E7E0000000000000010385410B0
:10E3C5001010101010543810007C00103854101024
:10E3D5001010101010101000001010101010101058
:10E3E5001010543810000000000010207E2010008E
:10E3F500000000000000000008047E040800000082
:10E405000000000000000202020202027E0000007D
:10E415000000000000247E24000000000000000031
:10E4250000101038383C7E7EFF000000000000FF21
:10E435007E7E3C383810100000000000000000000F
:10E44500000000000000000000080808080808088F
:10E455000008080000002424242400000000000017
:10E465000000000000909048FE4824FF241212008E
:10E475000000083C0A0A0A0C182828281E08000073
:10E4850000864929291668949492610000000018B5
:10E495002424140C8B917163FE0000000808080801
:10E4A50000000000000000000000603008080404BF
:10E4B5000404040808306000060C101020202020F9
:10E4C5002010100C060000080866142C240000001B
:10E4D50000000000000000000808087F0808080088
:10E4E50000000000000000000000001818100800DF
:10E4F5000000000000007E00000000000000000099
:10E505000000000000000018180000004020202036
:10E51500101018080804040402000018244242429E
:10E52500424242241800000000101E101010101066
:10E535001010FE000000001E20202010100804020C
:10E545003E000000003C40404038404040403C0018
:10E555000000002030282824227E202020000000F2
:10E56500007C0404041C604040403C00000000386E
:10E575000402023A4642424438000000007E402030
:10E5850020100808080404000000003C4242221C38
:10E59500244242423C000000001C224242625C4090
:10E5A50040201C00000000000000181800000018A2
:10E5B50018000000000000001818000000181810CE
:10E5C5000800000000004030080608304000000048
:10E5D50000000000007E00007E000000000000003A
:10E5E5000000020C1060100C02000000003E4240CA
:10E5F50020100808000808000000003C4672494940
:10E605004969DB223C000000000010182824244240
:10E615007E428100000000003E4242221E2242420C
:10E625003E00000000007C020101010101027C00A6
:10E63500000000001F214141414141211F00000010
:10E6450000007E0202023E0202027E00000000007F
:10E655007E0202023E0202020200000000007C026D
:10E665000101017141427C0000000000424242422A
:10E675007E4242424200000000003E0808080808A9
:10E6850008083E00000000003C202020202020201B
:10E695001E00000000004222120A060A1222420051
:10E6A5000000000002020202020202027E000000D7
:10E6B5000000636363555555494141000000000062
:10E6C5004246464A4A5252624200000000001C225D
:10E6D5004141414141221C00000000003E424242AE
:10E6E500621E02020200000000001C22414141415D
:10E6F50041221C60C00000001E2222221E1232226E
:10E705004200000000007C020206186040403E0006
:10E71500000000007F080808080808080800000035
:10E72500000042424242424242423C000000000098
:10E73500814242222414140808000000000081814F
:10E74500C9595A5A666624000000000081422418FF
:10E755001818244281000000000081422214180884
:10E7650008080800000000007F402010080402018E
:10E775007F00000078080808080808080808080845
:10E785007800020404040808181010202020400016
:10E795001E10101010101010101010101E00001078
:10E7A5001018282824444200000000000000000042
:10E7B50000000000000000FF000010200000000025
:10E7C5000000000000000000000000003C40407C0C
:10E7D5004242FC000000020202023A464242424620
:10E7E5003A000000000000007804020202047800EC
:10E7F5000000404040405C62424242625C000000D2
:10E80500000000003C44427E02027C0000007008CB
:10E8150008087E0808080808080000000000000035
:10E825007C62424242625C40403C020202023A463D
:10E835004242424242000000181800001E1010100B
:10E84500101010000000303000003C202020202057
:10E855002020201E0202020222120A061A2242006B
:10E8650000001E10101010101010101010000000E5
:10E87500000000006D5B494949494900000000005E
:10E8850000003A46424242424200000000000000B9
:10E895001C22414141221C000000000000003A46B4
:10E8A500424242463A020202000000005C624242D5
:10E8B50042625C404040000000003A26020202022B
:10E8C50002000000000000003C02061820201E0087
:10E8D5000000000004047F04040404047800000020
:10E8E500000000004242424242625C00000000001B
:10E8F50000008142422214140800000000000000BC
:10E9050081915A5A66242400000000000000422428
:10E91500181818244200000000000000814242241B
:10E92500241818080C07000000007F2010080402B6
:10E935007F0000007008080808080608080808088D
:10E945007000101010101010101010101010100082
:10E955000E10101010106010101010100E00000096
:10E96500000000869961000000000000000000081A
:10E975001C22414141417F00000000007C02010151
:10E98500010101027C102030002400004242424275
:10E9950042625C000000201000003C44427E0202FE
:10E9A5007C000000182400003C40407C4242FC00F2
:10E9B5000000002400003C40407C4242FC00000076
:10E9C500081000003C40407C4242FC00000010283A
:10E9D50010003C40407C4242FC000000000000006A
:10E9E50078040202020478081018182400003C4438
:10E9F500427E02027C000000004800003C44427E4A
:10EA050002027C000000081000003C44427E020225
:10EA15007C000000002400001E10101010101000D3
:10EA25000000182400001E10101010101000000027
:10EA3500081000001E101010101010000000240017
:10EA45001018282424427E42810000000814081C66
:10EA5500143422227E438100000020107E0202022F
:10EA65003E0202027E00000000000000778888FE5A
:10EA75000909F60000000000F018181474121E129F
:10EA8500F1000000182400001C22414141221C0015
:10EA95000000002400001C22414141221C0000000E
:10EAA500040800001C22414141221C0000001824DA
:10EAB50000004242424242625C000000040800003D
:10EAC5004242424242625C00000000240000814252
:10EAD5004224241818080C0724001C2241414141F6
:10EAE50041221C000000240042424242424242426E
:10EAF5003C000000000000007E63514945221F00D4
:10EB0500000000700808081C080808047C000000C4
:10EB150000005C226151494543221D0000000000B0
:10EB25000000412214081422410000007008080862
:10EB35003C080808080808080807201000003C40A1
:10EB4500407C4242FC000000201000001E10101006
:10EB5500101010000000201000001C22414141222D
:10EB65001C000000201000004242424242625C004C
:10EB75000000483400003A4642424242420000004A
:10EB850058344246464A4A52526242000000003C0E
:10EB95002038247C0000000000000000001C222218
:10EBA500221C000000000000000000000000101002
:10EBB500001010080402427C003C425A5A423C00B4
:10EBC5000000000000000000000000007F40400041
:10EBD5000000000000432232120AF8844632F10098
:10EBE500000000432212120A68544AFA410000004C
:10EBF50000000000080800080808080808080000C8
:10EC05000000482412122448000000000000000003
:10EC15001224484824120000000049000049000061
:10EC25004900490000490000924900924900924973
:10EC3500920049920049FF4949FF4949FF49FF4967
:10EC450049FF494910101010101010101010101025
:10EC550010101010101010101F10101010101010A0
:10EC650010081018282424427E4281000000182430
:10EC75001018282424427E42810000000810101834
:10EC8500282424427E4281000000003C42B985854B
:10EC95008585B9423C00000028282828282F202FE8
:10ECA50028282828282828282828282828282828DF
:10ECB5002828282800000000003F202F2828282881
:10ECC500282828282828282F203F00000000000099
:10ECD500001078141212121214781000000000812E
:10ECE500422414083E083E08080000000000000009
:10ECF50000001F1010101010101010101010101020
:10ED0500F000000000000000101010101010FF00AF
:10ED1500000000000000000000000000FF101010BF
:10ED250010101010101010101010F01010101010FE
:10ED35001010000000000000FF00000000000000AF
:10ED4500101010101010FF10101010101010483473
:10ED550000003C40407C4242FC0000005834101842
:10ED6500282424427E42810000002828282828E8FB
:10ED750008F80000000000000000000000F808E8A6
:10ED85002828282828282828282828EF00FF0000D8
:10ED9500000000000000000000FF00EF28282828E0
:10EDA50028282828282828E808E82828282828287E
:10EDB5000000000000FF00FF000000000000282800
:10EDC500282828EF00EF2828282828280000413E79
:10EDD500222222223E4100000000170C16203C6230
:10EDE500414141221C00000000003E4282828F8288
:10EDF50082423E00000018247E0202023E02020208
:10EE05007E00000024007E0202023E0202027E0015
:10EE1500000010207E0202023E0202027E00000077
:10EE2500000000001E10101010101000000020102F
:10EE35003E080808080808083E00000018243E0897
:10EE45000808080808083E00000024003E080808D5
:10EE5500080808083E0000001010101010101F00D0
:10EE6500000000000000000000000000F01010107D
:10EE750010101010FFFFFFFFFFFFFFFFFFFFFFFF59
:10EE8500FFFF00000000000000FFFFFFFFFFFFFF86
:10EE950010101010100000001010101010000810B5
:10EEA5003E080808080808083E000000FFFFFFFFAD
:10EEB500FFFFFF0000000000000020101C22414160
:10EEC500414141221C0000001C2222221212224232
:10EED50082827200000018241C22414141414122D6
:10EEE5001C00000008101C224141414141221C0028
:10EEF5000000483400001C22414141221C00000052
:10EF050058341C224141414141221C0000000000AF
:10EF150000004242424242665A02020202020202D4
:10EF25003A46424242463A020202000002023E428C
:10EF350042423E020200000020104242424242424A
:10EF450042423C00000018244242424242424242B0
:10EF55003C000000102042424242424242423C00F4
:10EF650000002010000081424224241818080C07D4
:10EF75002010814222141808080808000000FF002C
:10EF85000000000000000000000000001008000064
:10EF9500000000000000000000000000000000006C
:10EFA5007E000000000000000000000008087F0847
:10EFB50008007F00000000000000000000000000C5
:10EFC50000FF00FF00874423241768544CFA4100D2
:10EFD5000000007E4F4F4F4E48484848484848007B
:10EFE500007804041C34444C386040443C00000064
:10EFF50000001818007F001818000000000000002D
:10F0050000000000000000081018000814080000A7
:10F0150000000000000000002400000000000000C7
:10F0250000000000000000000000000018180000AB
:10F035000000000000181010101000000000000073
:10F045000000003C2018203C0000000000000000EB
:10F05500003C2010083C00000000000000000000FB
:10F0650000007E7E7E7E7E7E7E0000000000000029
:10F07500000000000000000000000000000000008B
:10F0850000000E111B111F0E00000E151F111F0E83
:10F0950000000A1F1F1F0E04000004040E1F0E04AB
:10F0A5000400040E041F15040E00040E1F1F150492
:10F0B5000E0000000000000000000000000000003D
:10F0C500000000000000000000000000000000003B
:10F0D500000018180E1111110E000E1111110E0459
:10F0E5000E040000000000000000181E12121A1B7A
:10F0F500030000150E1B0E1500000001071F070178
:10F10500000000101C1F1C100000040E0404040E57
:10F115000400000A0A0A000A00000E0B0B0A0A0A7C
:10F125000A000C02040A040806000000001E1E0066
:10F135000000040E040E04000E00040E0404040472
:10F14500040004040404040E04000000081E080062
:10F1550000000000041E0400000000000202021E60
:10F16500000000000A1F0A0000000004040E0E1F24
:10F175000000001F0E0E0404000000000000000047
:10F18500000004040404000400000A0A0000000052
:10F19500000000141F0A1F050000040E06040C0ED3
:10F1A500040012150E0E15090000040A06150916AD
:10F1B500000004040000000000001804020202041C
:10F1C50018000304080808040300040A040A0000E0
:10F1D5000000000000040E04000000000000000410
:10F1E50004020000000E0000000000000000000402
:10F1F500000010080804040202000C121212120C7E
:10F20500000004060404040E000006080804020EAB
:10F2150000000608060808060000080C0A1E080873
:10F2250000000E020608080600000C020E12120C61
:10F2350000001E100804040400000C120C12120C2D
:10F2450000000C12121C100C000000000400000449
:10F255000000000004000004040200100806081065
:10F26500000000001E001E00000000020418040239
:10F2750000000E100804000400000C1219151D01F1
:10F285001E0000040A0A1F110000000E0A060A0EDD
:10F295000000001C0202021C0000000E1212120ED9
:10F2A5000000000E020E020E0000000E020E020209
:10F2B5000000001C021A121C00000012121E12127D
:10F2C5000000000E0404040E0000000E08080806E5
:10F2D500000000120A060A12000000020202021EC5
:10F2E500000000111B15151100000012161A12124C
:10F2F5000000000E1111110E0000000E120E020288
:10F305000000000E1111110E081000060A060A125F
:10F315000000000C020408060000001F0404040499
:10F32500000000121212120C0000001212120C0C36
:10F335000000001115150A0A000000110A040A113F
:10F34500000000110A0404040000001E100C021E37
:10F3550000000C04040404040C0001020204040867
:10F3650008000604040404040600040A0A11110036
:10F3750000000000000000001F0002040000000063
:10F385000000000006080E1E000002020E12120EFA
:10F39500000000000C02020C000008080E09090E0E
:10F3A50000000000040E020C000018041E040404F2
:10F3B500000000001C121E100E0002020A16121296
:10F3C5000000040006040404000008000E080808F4
:10F3D500060002020A060A120000060404040404D8
:10F3E50000000000151F1515000000000A16121276
:10F3F500000000000C12120C000000000E12120E8C
:10F40500020000000E09090E080000000A060202AB
:10F41500000000000C060806000000041E04040895
:10F425000000000012121A140000000012120C0C49
:10F435000000000015150E0A00000000120C0C1249
:10F445000000000012120C0C070000000E0C020E4A
:10F45500000008040402040408000404040404046D
:10F465000400020404080404020000000016090058
:10F47500000000040A0A0A0E0000001C0202021C19
:10F485000804120012121A1400001008040E020CCF
:10F4950000000C1206080E1E00000A0006080E1ECB
:10F4A5000000010206080E1E0000040A06080E1ED2
:10F4B500000000000C02020C08040C12040E020CE1
:10F4C50000000A00040E020C00000102040E020CEA
:10F4D50000000A000604040400000C1206040404DB
:10F4E500000001020604040400000A040A0A1F11B0
:10F4F5000000040A040A1F110000100E020E020E7D
:10F50500000000000B1C07190000001C0A1A0F1947
:10F51500000006090C12120C000012000C12120C4D
:10F52500000001020C12120C0000060912121A1436
:10F535000000020412121A140000120012120C0C20
:10F545000700110E1111110E000009121212120CF2
:10F55500000000100C1A160C020000040206030E2F
:10F565000000100E1915130E01000000120C0C12EC
:10F5750000000804040E04040200100806080E1E0C
:10F585000000100806040404000010080C12120CF8
:10F595000000100812121A1400001E000A1612129A
:10F5A50000001F12161A1212000006080E0A0E009D
:10F5B5000000040A0A0A040000000004000404080C
:10F5C50006000E1D1D151D0E00000000000E08088A
:10F5D5000000130A1E140A190000130A0A141A114E
:10F5E5000000000004000404040000140A050A14C5
:10F5F500000000050A140A05000015001500150095
:10F605001500150A150A150A150A1F151F151F15C8
:10F615001F15040404040404040404040407040476
:10F62500040408040A0A1F1100000C12040A1F1121
:10F63500000002040A0A1F1100000E111D151D11FC
:10F645000E000A0A0B080B0A0A0A0A0A0A0A0A0A1B
:10F655000A0A00000F080B0A0A0A0A0A0B080F001B
:10F66500000000040E020E04000000110A040E043E
:10F67500000000000007040404040404041C000046
:10F6850000000404041F000000000000001F040423
:10F6950004040404041C040404040000001F000006
:10F6A50000000404041F04040404160906080E1EC1
:10F6B50000001609040A1F1100000A0A1A021E009A
:10F6C500000000001E021A0A0A0A0A0A1B001F008F
:10F6D500000000001F001B0A0A0A0A0A1A021A0A79
:10F6E5000A0A00001F001F0000000A0A1B001B0A6F
:10F6F5000A0A00110E0A0E1100000F040E09090670
:10F705000000000E1217120E00000E0E020E020E61
:10F715000000110E020E020E0000010E020E020E76
:10F7250000000000060404040000100E0404040E8A
:10F7350000000E0E0404040E0000110E0404040E55
:10F74500000004040407000000000000001C04047D
:10F7550004041F1F1F1F1F1F1F1F000000001F1F66
:10F765001F1F0404040000040404010E0404040E15
:10F7750000001F1F1F1F00000000100E1111110EA9
:10F785000000040A0A0A120A00000E0E1111110ED9
:10F795000000010E1111110E000016090C12120CB9
:10F7A50000000F0E1111110E0000000012121A16A2
:10F7B500020002020E12120E020000020E120E02CA
:10F7C500000010090909090600001E121212120C88
:10F7D500000001121212120C0000100812120C0C7B
:10F7E500030008150A04040400001F0000000000BF
:10F7F500000008040000000000000000000E0000EA
:10F8050000000000040E040E000000000000001FB0
:10F81500001F130B0A171A1100000E0B0B0A0A0A18
:10F825000A000C02040A040806000004000E000485
:10F83500000000000000000004020C12120C000081
:10F8450000000A00000000000000000000040000A5
:10F855000000060404040E00000006080608060061
:10F865000000060804020E00000000001E1E1E1EF9
:10F875000000000000000000000000000000000083
:10F88500040A0E0A0400040E0A0E0400000A0E0EF5
:10F89500040000040E0E0400040E0E040E00040401
:10F8A5000E040E0000000000000000000000000033
:10F8B500000000000000000000000000000C080629
:10F8C5000600040A040E0400000000000000040CF9
:10F8D5000A080400040E0A0E040002060E060200C1
:10F8E500080C0E0C0800040E040E04000A0A0A0097
:10F8F5000A000008040404040404040402000000CF
:10F9050000000E00040E040E040E040E0404040090
:10F915000404040E040000040F04000000020F029A
:10F9250000000000020E0000000A0E0A000000049C
:10F935000E0E0000000E0E04000000000000000086
:10F945000404040004000A0A000000000A0E0A0E5E
:10F955000A00040C060C0604020804020800040A46
:10F965000C0A0E0006020000000004020202040058
:10F975000204040402000A040E040A0000040E0432
:10F98500000000000000060200000E00000000005C
:10F99500000004000808040202000C0A0A0A060016
:10F9A500040604040E00060804020E0006080408F6
:10F9B5000600080A0E0808000E02060806000402E2
:10F9C500060A04000E080C040400040A040A0400D4
:10F9D500040A0C08040000000400040000000400F0
:10F9E500060208040204080000000E000E000204CE
:10F9F500080402000608040004000E0A0A020E00AC
:10FA0500040A0E0A0A00060A060A06000C02020289
:10FA15000C00060A0A0A06000E0206020E000E0275
:10FA2500060202000C020A0A0C000A0A0E0A0A0063
:10FA35000E0404040E000808080A04000A0A060A4F
:10FA45000A00020202020E000A0E0E0A0A000A0E3F
:10FA55000A0A0A00040A0A0A0400060A0602020043
:10FA6500040A0A0E0C00060A060A0A000C020E0811
:10FA750006000E04040404000A0A0A0A0E000A0A13
:10FA85000A0A04000A0A0E0E0A000A0A040A0A00F3
:10FA95000A0A040404000E0804020E00060202020B
:10FAA5000600020204080800060404040600040A0D
:10FAB5000000000000000000000F06040000000028
:10FAC50000000C0A0E000202060A060000000C02E5
:10FAD5000C0008080C0A0C0000000E060C000804B7
:10FAE5000E04040000000E0A080E0202060A0A00AF
:10FAF50004000404040004000404040602020A06C7
:10FB05000A0004040404040000000E0E0A000000AC
:10FB1500060A0A000000040A04000000060A06029C
:10FB250000000C0A0C0800000602020000000C048C
:10FB3500060000040E040C0000000A0A0E00000076
:10FB45000A0A040000000A0E0E0000000A040A005A
:10FB550000000A0A0402000006040C000C04060456
:10FB65000C0004040404040006040C0406000A0541
:10FB75000000000000040A0E00000C02020E040240
:10FB85000A000A0A0C0008040E060C00040A0C0AF6
:10FB95000E000A000C0A0E0002040C0A0E000400F6
:10FBA5000C0A0E00000E020E0406040A0E060C00D6
:10FBB5000A000E060C0002040E060C000A000404DE
:10FBC5000400040A000404000204000404000A04FA
:10FBD5000A0E0A0004040A0E0A0008040E060E00A6
:10FBE50000000C0E06000C060E060E00040A040AA0
:10FBF50004000A00040A04000204040A0400040ABA
:10FC0500000A0E0002040A0A0E000A000A0A04028B
:10FC15000A040A0A04000A000A0A0E00040E020E6B
:10FC2500040008040E040E000A0E040E040000066B
:10FC3500060A0A000C040C04060008040C0A0E004F
:10FC450008040004040008040E0A0E000804000A53
:10FC55000E000E000E0A0A000E000A0E0A000C0A1B
:10FC65000E000E00040A04000E00040004020C003D
:10FC7500000E02020000000704040000020A040A44
:10FC85000C00020A040E0800040004040400000A23
:10FC9500050A000000050A0500000208020802081E
:10FCA5000A050A050A050D070D070D0704040404D6
:10FCB50004040404070404040407040704040A0AEA
:10FCC5000B0A0A0A00000F0A0A0A000704070404BF
:10FCD5000A0B080B0A0A0A0A0A0A0A0A000F080B85
:10FCE5000A0A0A0B080F00000A0A0F0000000407A1
:10FCF5000407000000000704040404040C000000CD
:10FD050004040F00000000000F04040404040C04A4
:10FD1500040400000F00000004040F040404040C94
:10FD2500040C04040A0A0A0A0A0A0A0A020E000056
:10FD3500000E020A0A0A0A0B000F0000000F000B52
:10FD45000A0A0A0A020A0A0A000F000F00000A0B33
:10FD5500000B0A0A040F000F00000A0A0F0000003A
:10FD6500000F000F040400000F0A0A0A0A0A0E0019
:10FD75000000040C040C0000000C040C040400003A
:10FD85000E0A0A0A0A0A0B0A0A0A040F000F0404DB
:10FD950004040700000000000C0404040F0F0F0FFB
:10FDA5000F0F0000000F0F0F0303030303030C0CD9
:10FDB5000C0C0C0C0F0F0F00000000000E060E00BF
:10FDC500040A060A06020E0A020202000E0A0A0ABE
:10FDD5000A000E0204020E0000000C0A04000000D6
:10FDE5000A0A0E020008060404000E040A040E00A6
:10FDF500040A0E0A040000040A0A0A000C02040A96
:10FE0500040000000E0A0E00040E0A0E04000C0287
:10FE15000E020C00040A0A0A0A000E000E000E006B
:10FE2500040E04000E00060806000E000C020C006D
:10FE35000E00000804040404040404040200040081
:10FE45000E000400000A050A0500040A040000006B
:10FE550000040E0400000000040000000C04040669
:10FE650004000E0A0A000000060402060000000055
:10FE7500060600000000000000002C632C632C63C4
:10FE85002C63FFFFFFFF4D6B4D6B1CE71CE7139DBC
:10FE9500139D2C632C632C632C63139D139D139D61
:10FEA500139D7DEF7DEF7DEF7DEF2C632C632C6340
:10FEB5002C63FFFFFFFF4D6B4D6B1CE71CE7139D8C
:10FEC500139D2C632C632C632C63139D139D139D31
:10FED500139D7DEF7DEF7DEF7DEF2C632C632C6310
:10FEE5002C63FFFFFFFF4D6B4D6B1CE71CE7139D5C
:10FEF500139D7FF000050008000000FF0000007F53
:10FF0500F800040006000000FF0000007FE2000882
:10FF1500000E000000FF0000007FAE0010001A0078
:10FF25000000FF000000FF01990000000BB8A3FFCF
:10FF350001860000000000792323232323232323A4
:10FF4500232323232323232323232323232323237C
:10FF55002323232323230D0A0054656D70657261E5
:10FF650074757265206F757473696465203D200032
:10FF7500436F6E66696775726174696F6E20646F31
:10FF85006E650D0A00416972207072657373757232
:10FF950065203D2000496E69742073656E736F722C
:10FFA500732E2E2E0054656D7065726174757265C1
:10FFB500203D200048756D6964697479203D2000F5
:10FFC50025346C752E2530326C7500434F32203D3B
:10FFD500200025352E30326600252E306600252E70
:10FFE5003266006D62617200253464005248004338
:0BFFF5004F002D0032004300460000CA
:020000040020DA
:08000000FFFFFFFFFFFFFFFF00
:020000040030CA
:0E000000FF28183CFF3F81FF0FC00FE00F40AC
:00000001FF
